:020000040000FA
:10000000000000008EEF0EF01200800E016EFE0E5A
:1000100089D9010E87D9750E106E300EB9D1016ADB
:10002000018E1F6EFE0E7ED91F507CD1056A800E98
:10003000326E00D0176A186A196A1A6A069A7DD950
:10004000D30FD8B4068A2D0FC60FF9E20A0FF7E3D3
:10005000136E126A116A106A0A0E0F6E4FEC02F0EC
:1000600013500F24176E1050186E000ED8B0010EEA
:1000700018261150196E000ED8B0010E1926125014
:100080001A6E000ED8B0010E1A26050605E055D9E5
:10009000C60F02E20A0FDCE206AA0BD0171E181EDA
:1000A000191E1A1E172AD8B4182AD8B4192AD8B477
:1000B0001A2A1750120030D803D0056A176E186A32
:1000C00000960550D8B40086050E046E270E146EF7
:1000D000100E0CD8030E146EE80E08D8146A640EC5
:1000E00005D8146A0A0E02D8175007D0136E18509C
:1000F000106E17500F6E81D90F500F6E044E009680
:10010000055002E0045C07E20F50D8A4009600B648
:1001100002D0300F07D1120018AE1200175018107D
:10012000D8B41200171E181E174A182A2D0EFAD01E
:10013000346E23AE02D02D0EF5D8253E04D0243ED9
:1001400002D0234A232A2A6A2B6A2C6A2D6A238E1C
:100150006A0E2226D8902332243225322D322C32B8
:100160002B322A32223EF6D72550225C2526225EEB
:100170002450235C2426235E056A38D82E0ED2D85C
:10018000356AD8902A34256E2B34246E2C34236E95
:100190002D34226E3536D890253624362336223635
:1001A00035362A5025262B50D8B02B3C24262C50EF
:1001B000D8B02C3C23262D50D8B02D3C2226D8B0C8
:1001C000353ED890253624362336223635363550FE
:1001D000300FA8D825C02AF024C02BF023C02CF063
:1001E00022C02DF0342ECCD7D890120000960550A6
:1001F00003E100860A0E056E25C012F024C011F03E
:1002000023C010F022C00FF0046A1A6A196A186A33
:100210000A0E176EC7D8042A0450055CF6E1175081
:10022000D8A4009600A602D0052C03D01750300F9A
:1002300079D8052EE1D71200176E0450D8B41200F9
:1002400017C0E9FF18C0EAFFEF50D8B412006AD80F
:10025000174A182A0406F1D7A66AA68E0900F55097
:1002600002E002D8FBD712001C6E8998899A9298F6
:10027000929AF00E92161C5000B21ED03A0E106EDA
:10028000980E86D8330E1B6E29D8130E106E880E6A
:100290007FD824D8640E7BD821D8640E78D8220E5B
:1002A0001B6E1CD8280E07D80C0E05D8060E03D8D6
:1002B00000821C5001D000801B6E00A009D0899ADA
:1002C00003080AE309D8090E106EC40E61D81200A3
:1002D0000080FE0814E0898A1B3A00A000908988FB
:1002E000F00E80161B500F0B8012000000D0899872
:1002F0001B3A000000D000B0F1D7320E48D81C5095
:1003000012009EAAFED7AE50D8801200A66AA68E12
:100310000900F55002E002D8FBD712009EA8FED7D4
:10032000AD6E120001BEA0D701B4F8D701A205D06E
:1003300001B003D001B2EE6E120032AE02D0EE5028
:1003400012003204DEE0A86EA66AA684550EA76EDF
:10035000AA0EA76EA682A6B2FED7A694A94AAA2A7A
:10036000A68E1200A96EA66AA680A850A94AAA2A3B
:10037000A68E1200146A136EFF0E1326142200D0EC
:10038000D8A01200030E106EE60E02D8F5D7106A40
:10039000FD0F0F6E01D00F06000000D0E86A105A62
:1003A000FAE21200266A276A286A296A210E156E67
:1003B00015D026362736283629361750265C185091
:1003C0002758195028581A50295808E3296E1750F1
:1003D000265E1850275A1950285AD8800F361036E2
:1003E00011361236152EE5D729C01AF028C019F09B
:1003F00027C018F02650176E1200186A176A100EE0
:10040000F36E1034173618361350175C1450185802
:1004100005E31350175E1450185AD8800F36103663
:10042000F32EEFD70F5012001E501818800BF46EE9
:100430001EAE05D01D1E1E1E1D2AD8B41E2A18AEC3
:1004400005D0171E181E172AD8B4182A136A0F6A67
:10045000106A146A185002E1175018E0100EF36E7B
:10046000D8901D361E36133614361850145C02E12F
:100470001750135C07E31750135ED8A014061850EA
:10048000145ED8800F361036F32EEAD7F4AE05D0BE
:100490000F1E101E0F2AD8B4102A0F50120012C0BF
:1004A00029F011C028F010C027F00FC026F0285006
:1004B0001702F3CF11F0F4CF12F027501802F350C7
:1004C0001126F450122226501902F3501126F4502E
:1004D000122229501702F350122628501802F35006
:1004E000122627501902F350122626501A02F350F2
:1004F000122626501702F3CF0FF0F4CF10F027503A
:100500001702F3501026F4501122000E122226502A
:100510001802F3501026F4501122000E122212007D
:100520000F6E10BE02D80F5012000F1E101E0F4A81
:10053000102A1200A66AA68E0900F55002E0EE6E9F
:10054000FBD71200E752E6CFEEFF02E0E82EFAD723
:100550001200F34E02D0E652FCD7E6CFEEFFE82EB3
:10056000FCD71200E466FED7F36EE552F32EFDD7FA
:10057000E6CFEEFFE82EFCD71200A66AA68EEE505C
:100580000900F55C02E1F566FAD71200A66AA68EAC
:10059000EE500900F55C03E1F566FAD7010C000C9A
:1005A000A66AA68EEE500900F55C03E1F566FAD75F
:1005B000000C010C296A2DC012F02CC011F02BC0C8
:1005C00010F02A500F6E05E02BAE03D02980800E6C
:1005D000101A10BE21D0010E125C000E1158000E30
:1005E00010587F0E0F5818E32D6A2C6A2B6A7F0E65
:1005F0002A6E12C031F011C030F010C02FF00FC0C1
:100600002EF07DEC07F02DC012F02CC011F02BC0A5
:1006100010F02AC00FF029820A0E2D6E890E2C6E62
:10062000340E2B6E7C0E2A6E12C031F011C030F0E9
:1006300010C02FF00FC02EF0E3EC07F012C031F025
:1006400011C030F010C02FF00FC02EF0E3EC07F017
:100650007C0E316E790E306E350E2F6E810E2E6E41
:10066000EFEC06F012C031F011C030F010C02FF0E6
:100670000FC02EF0E3EC07F012C031F011C030F0E3
:1006800010C02FF00FC02EF0E3EC07F03F0E316EDC
:10069000020E306E330E2F6E830E2E6EEFEC06F0D0
:1006A00012C031F011C030F010C02FF00FC02EF08A
:1006B000E3EC07F012C031F011C030F010C02FF0A1
:1006C0000FC02EF0E3EC07F0330E316E8C0E306E5F
:1006D0001E0E2F6E830E2E6EEFEC06F02DC016F060
:1006E0002CC015F02BC014F02AC013F012502D6E40
:1006F00011502C6E10502B6E0F502A6E12C031F01C
:1007000011C030F010C02FF00FC02EF0E3EC07F056
:100710001B0E316EE40E306E350E2F6E820E2E6E75
:10072000EFEC06F012C031F011C030F010C02FF025
:100730000FC02EF0E3EC07F012C031F011C030F022
:1007400010C02FF00FC02EF0E3EC07F0A40E316EB6
:10075000DB0E306E670E2F6E830E2E6EEFEC06F002
:1007600012C031F011C030F010C02FF00FC02EF0C9
:10077000E3EC07F012C031F011C030F010C02FF0E0
:100780000FC02EF0E3EC07F0330E316E8C0E306E9E
:100790001E0E2F6E830E2E6EEFEC06F02DC01AF09B
:1007A0002CC019F02BC018F02AC017F012C02DF081
:1007B00011C02CF010C02BF00FC02AF016C031F081
:1007C00015C030F014C02FF013C02EF0E3EC07F08A
:1007D0001AC031F019C030F018C02FF017C02EF039
:1007E0007DEC07F02DC031F02CC030F02BC02FF085
:1007F0002AC02EF029A20AD0DB0E2D6E0F0E2C6E11
:10080000490E2B6E7F0E2A6EEDEC06F029A002D069
:10081000800E2B1A2D501200010E176E36C019F0E3
:10082000368C1A6A176602D02BBE1A8E2B9E880E43
:100830002A60368A2DC00FF02CC010F02BC011F0AA
:100840002AC012F0830E316EF90E306E220E2F6E1A
:100850007F0E2E6EE3EC07F031EC08F02AA004D0F6
:100860002A2A000E2B222C22070E2A14186E030EA1
:10087000186404D0800E1A1A040E185E2D6A90ECCB
:1008800008F02A50166E6DE02DC013F02CC014F045
:100890002BC015F0316A0F0E306EC90E2F6E7E0E12
:1008A0002E6EE3EC07F00FC031F010C030F011C035
:1008B0002FF012C02EF0EFEC06F02DC00FF02CC080
:1008C00010F02BC011F02AC012F013C02DF014C08C
:1008D0002CF015C02BF016C02AF0316AA20E306E33
:1008E000DA0E2F6E6E0E2E6EE3EC07F00FC031F0B5
:1008F00010C030F011C02FF012C02EF0EFEC06F057
:100900002DC00FF02CC010F02BC011F02AC012F037
:1009100013C02DF014C02CF015C02BF016C02AF017
:10092000200E316EA20E306E850E2F6E5C0E2E6E76
:10093000E3EC07F00FC031F010C030F011C02FF021
:1009400012C02EF0EFEC06F02A50126E2E6E2B50D5
:10095000116E2F6E2C50106E306E2D500F6E316E4A
:100960000CD012502A6E2E6E11502B6E2F6E10501E
:100970002C6E306E0F502D6E316EE3EC07F02DC0F3
:1009800013F02CC014F02BC015F02AC016F018304C
:100990001818010B17184EE0CE0E316EF50E306EA2
:1009A0004C0E2F6E6F0E2E6EE3EC07F01A0E316EAA
:1009B000060E306EB60E2F6E750E2E6EEFEC06F034
:1009C00013C031F014C030F015C02FF016C02EF057
:1009D000E3EC07F0A50E316EAA0E306E2A0E2F6ED4
:1009E0007A0E2E6EFCD913C031F014C030F015C051
:1009F0002FF016C02EF0E3EC07F013C031F014C056
:100A000030F015C02FF016C02EF0E3EC07F013C045
:100A100031F014C030F015C02FF016C02EF02E6645
:100A20002E06DBD9369C316A306A2F6A7F0E2E6E15
:100A3000D6D956D0F90E316E680E306E360E2F6E46
:100A40006C0E2E6EE3EC07F0C00E316E070E306EAA
:100A5000D00E2F6E720E2E6EC2D913C031F014C09C
:100A600030F015C02FF016C02EF0E3EC07F0840E26
:100A7000316E880E306E080E2F6E780E2E6EAFD946
:100A800013C031F014C030F015C02FF016C02EF096
:100A9000E3EC07F0AB0E316EAA0E306E2F6E7C0EBB
:100AA0002E6E9DD913C031F014C030F015C02FF058
:100AB00016C02EF0E3EC07F00FC031F010C030F09C
:100AC00011C02FF012C02EF0E3EC07F0369C0FC0DF
:100AD00031F010C030F011C02FF012C02EF07FD9CD
:100AE000800E175202E018B21A1A1ABE2B1A19BC3D
:100AF000368C2D5012002BBEA6D02A52D8B4A4D0CA
:100B00002AC018F036C019F0368C7F0E2A6E316A72
:100B1000306A2F6A2E6E61D92DC00FF02CC010F0F4
:100B20002BC011F02AC012F0130E316ECB0E306EB6
:100B3000030E2F6E840E2E6E52D90FC031F010C0EE
:100B400030F011C02FF012C02EF0E3EC07F0BC0E15
:100B5000316E5A0E306E050E2F6E860E2E6E3FD9F8
:100B60000FC031F010C030F011C02FF012C02EF0C5
:100B7000E3EC07F0830E316E300E306E720E2F6E86
:100B8000850E2E6E2CD92DC013F02CC014F02BC066
:100B900015F02AC016F00FC02DF010C02CF011C0B7
:100BA0002BF012C02AF08E0E316ED70E306E6B0E07
:100BB0002F6E810E2E6EE3EC07F0B50E316E290E0E
:100BC000306E4E0E2F6E840E2E6E09D90FC031F08E
:100BD00010C030F011C02FF012C02EF0F4D9800EEA
:100BE000316E300E306E720E2F6E840E2E6EF7D870
:100BF00013C031F014C030F015C02FF016C02EF025
:100C00007CD90FC031F010C030F011C02FF012C0ED
:100C10002EF0D9D9316A306A2F6A7F0E2E6EDFD856
:100C200018B009D0F30E316E040E306E350E2F6EF3
:100C30007F0E2E6EC8D97F0E182618302A6E19BC6A
:100C400003D0369C01D0368A2D5012002A502E62D5
:100C5000000C2B502F62000C2C503062000C2D50D9
:100C60003162000C010C2F502B18396E39BE30D078
:100C70002FBE17D02E502A5CD8A0000CD8A4010C8F
:100C80002F502B5CD8A0000CD8A4010C30502C5C49
:100C9000D8A0000CD8A4010C31502D5CD8A0000CB9
:100CA000010C2A502E5CD8A0000CD8A4010C2B50AB
:100CB0002F5CD8A0000CD8A4010C2C50305CD8A01C
:100CC000000CD8A4010C2D50315CD8A0000C010CF4
:100CD0002BAE010C000C2F502B18396E39BE34D0BE
:100CE0002FBE19D02E502A5CD8A0000CD8A4010C1D
:100CF0002F502B5CD8A0000CD8A4010C30502C5CD9
:100D0000D8A0000CD8A4010C31502D5CD8A0000C48
:100D1000D8A4010C000C2A502E5CD8A0000CD8A43A
:100D2000010C2B502F5CD8A0000CD8A4010C2C5027
:100D3000305CD8A0000CD8A4010C2D50315CD8A098
:100D4000000CD8A4010C000C2BAE010C000C2B5095
:100D50002F18396E39BE34D02BBE19D02A502E5CD4
:100D6000D8A0000CD8A4010C2B502F5CD8A0000CEC
:100D7000D8A4010C2C50305CD8A0000CD8A4010CD5
:100D80002D50315CD8A0000CD8A4010C000C2E50C2
:100D90002A5CD8A0000CD8A4010C2F502B5CD8A042
:100DA000000CD8A4010C30502C5CD8A0000CD8A4A6
:100DB000010C31502D5CD8A0000CD8A4010C000C03
:100DC0002FAE010C000C316A306A7E0E2E6E800E42
:100DD0002BAE000E2F6E03D844D1800E2F1A2E504A
:100DE0002A5C356E11E2356C2A502EC02AF02E6E28
:100DF0002B502FC02BF02F6E2C5030C02CF0306EAB
:100E00002D5031C02DF0316E1A0E356074D02E5237
:100E100072E0346A2B50386E2F18376E2B8E2F8E5F
:100E2000080E355E08E331C034F030C031F02FC019
:100E300030F02F6AF5D7352607E0D8902F323032C0
:100E400031323432352EF9D737AE33D031502D5EB2
:100E500030502C5A2F502B5A07E2D880000E2D56B6
:100E60002C562B56800E381A346C04E02D06000EDA
:100E70002C5A2B5A040E356E2B660DD02CC02BF03D
:100E80002DC02CF034C02DF0346A080E2A5E29E300
:100E9000352EF2D726D02BBE08D0D89034362D363A
:100EA0002C362B362A2EF7D71CD034AE22D0346AFB
:100EB0000FD031502D2630502C222F502B2206E3FC
:100EC0002B322C322D3234322A4A0DD034AE11D08E
:100ED0002D3E0FD02C3E0DD02B3E0BD0D8802D9028
:100EE000EFD72A6A02D036822A682D6A2C6A800ED1
:100EF0002B6E38AE2B9E2D5012002B50286E2F18C3
:100F0000376E2E5051E02A5252E02A5E7F0E03E2E5
:100F10002A2603E24BD02A264CE22DC026F02CC014
:100F200027F0288E2F8E180E386E2D6A2C6A2B6AA9
:100F30000BD03150265C3050275811E3276E286AB9
:100F40003150265E0BD004E22F50285CF2E007E31C
:100F50003150265E3050275A2F50285AD8802D36CF
:100F60002C362B36263627362836382EECD72BBE95
:100F700007D02A521BE037322A06382A3736E3D701
:100F800007E23150265E3050275A2F50285A17E377
:100F90002D3E15D02C3E13D02B3E11D02B322C32AF
:100FA0002D322A3E0CD005D0368604D036842A6AEB
:100FB00002D036822A682D6A2C6A800E2B6E37AEDC
:100FC0002B9E2D5012002B50286E2F18376E2A5052
:100FD000D8A42E503AE02A267E0E03E32A5E03E3CD
:100FE00036D02A5E31E32DC026F02CC027F0288EA3
:100FF0002F8E2D6A2C6A2B6A180E386E28322732F3
:10100000263206E331502D2630502C222F502B2231
:101010002B322C322D32382EF1D72BBE07D02D3665
:101020002C362B362A5210E02A06283416E32D3EA1
:1010300014D02C3E12D02B3E10D0D8802B322C3224
:101040002D322A3E0AD003D036842A6A02D0368254
:101050002A682D6A2C6A800E2B6E37AE2B9E2D507F
:1010600012002AC038F02B502DC02BF02D6E2D36DB
:1010700038322D32366A2D36383602E33684367EE3
:1010800006E13680386A2D6A2C6A2B6A0BD0382824
:1010900003E0D8802D3206D0D8902D3202E136827E
:1010A00001D0368636B604D036A20FD036B407D07B
:1010B0007F0E2D6EFF0E2C6E2B6E2A6E23D0800EAF
:1010C0002D6E01D02D6A000EF6D736B0FBD72A6AF6
:1010D0009F0E3860EBD77E0E3864F4D79E0E385CD6
:1010E00007E0D8902D322C322B322A32382AF6D70C
:1010F00036A408D0D880000E2A562B562C562D56D2
:101100002DAEE0D72A501200000E2BBEFF0E2C6E23
:101110002D6E06D02A6E2B6A2C6A2D6A379E0AD055
:10112000379E2DAE07D0D880000E2A562B562C564F
:101130002D56378E960E386E2D5209E0080E382641
:101140002BC02AF02CC02BF02DC02CF011D02C522B
:101150000FE1080E385E2B5007E1080E385E2A506A
:1011600002E12D5010D02A6A2C6E2AC02BF02A6A78
:101170002CBE06D0D8902A362B362C363806F8D717
:1011800037AE2C9E38502AC02DF02A6E2C502BC022
:101190002CF02B6E1200202020205049433138467D
:1011A000343532352020202020200000202020202F
:1011B000416E74656E6E6120526F746F72202020D4
:1011C000000020436F6E74726F6C6C6572207665E0
:1011D000722E0000416E74656E6E6120526F746FE6
:1011E0007220436F6E74726F6C6C657220762E2065
:1011F000000056657273696F6E2000005061726B5B
:10120000696E6720415A3D00417A696D75746820A6
:101210006F66667365743D200000417A696D757470
:1012200068206F666673657420736176656400007C
:10123000456C65766174696F6E206F666673657460
:101240003D200000456C65766174696F6E206F66A5
:101250006673657420736176656400002D2D2D2DF5
:101260002D2D2D2D2D2D2D2D2D2D434F4D4D414E01
:1012700044204C4953542D2D2D2D2D2D2D2D2D2D0C
:101280002D2D2D2D00003F202048656C70205465C9
:101290007874000041202043572F43435720526F5A
:1012A000746174696F6E2053746F70004220204126
:1012B0006E74656E6E6120446972656374696F6EE9
:1012C00020454C00432020416E74656E6E612044C1
:1012D0006972656374696F6E20415A004332204120
:1012E0006E74656E6E6120446972656374696F6EB9
:1012F00020415A26454C0000442020446F776E2040
:10130000446972656374696F6E20526F74617469A9
:101310006F6E000045202055502F444F574E2044FB
:101320006972656374696F6E20526F746174696F5E
:101330006E2053746F700000462020536574206D3A
:101340006178696D616C20706F736974696F6E206C
:10135000696E20617A696D7574683A2046616161D1
:101360000000462120536176652063757272656EB8
:101370007420706F736974696F6E206173206D6182
:1013800078696D616C20706F736974696F6E0000AD
:10139000463F2053686F77206D6178696D616C20DE
:1013A000706F736974696F6E20696E20617A696D00
:1013B00075746800472020536574204F6666736516
:1013C0007420496E20454C3A204765656500473FCB
:1013D0002053686F77204F666673657420436F6E85
:1013E0007374616E7420666F7220454C0000482053
:1013F0002048656C70207465787400004920205383
:10140000686F7720706172616D657465727300003A
:101410004A442053657420426565706572206F6E82
:10142000202D204469726563742043757272656E65
:1014300074004A46205365742042656570657220C9
:101440006F6E202D204672657175656E63790000A0
:101450004A4E2053657420426565706572206F6640
:1014600066004B2020416E74656E6E612044697287
:10147000656374696F6E2053657474696E67204983
:101480006E20454C3A204B65656500004C2020439A
:101490006F756E74657220436C6F636B77697365EB
:1014A00020526F746174696F6E004D2020416E741C
:1014B000656E6E6120446972656374696F6E205356
:1014C000657474696E6720496E20415A3A204D61F7
:1014D000616100004F20204F666673657420496E7D
:1014E00020415A004F3F2053686F77204F66667344
:1014F000657420436F6E7374616E74004F212053C6
:101500006176652063757272656E7420706F7369A1
:1015100074696F6E2061732053544F5020706F7345
:101520006974696F6E005020205061726B696E673C
:1015300020546F3A2050616161206565650050213B
:1015400020536176652063757272656E7420706FCA
:10155000736974696F6E206173207061726B696E5C
:10156000672076616C7565730000503F2053686F8B
:1015700077207361766564207061726B696E672095
:1015800076616C7565730000512020507265636947
:1015900073696F6E20302E31202D20302E35202D96
:1015A00020312E30206465670000522020436C6F8C
:1015B000636B7769736520526F746174696F6E0035
:1015C000532020416C6C2053746F700055202055BF
:1015D0007020446972656374696F6E20526F746124
:1015E00074696F6E0000562020536F6674766172C6
:1015F000652056657273696F6E00572020416E74C6
:10160000656E6E6120446972656374696F6E205304
:10161000657474696E673A2057616161206565651C
:1016200000005920204543484F204F4E202F204F87
:10163000464600005A2020537769746368207A6513
:10164000726F20706F736974696F6E20746F204EB3
:101650006F7264202F20536F75746800262020530A
:101660006574206D6178696D756D20656C65766156
:1016700074696F6E2028313830202D20666C6970B7
:10168000206F6E3B203930202D20666C6970206FF2
:1016900066662900252020456C65766174696F6E49
:1016A00020636F6E74726F6C204F4E202F204F4658
:1016B00046002A20204D61782E20656C6576617485
:1016C000696F6E20666F72206F7665727475726EC8
:1016D000696E6700232020456D756C6174696F6EBB
:1016E000206F6620475332333241202F2047533238
:1016F000333242003C2020417A696D757468206362
:10170000616C6962726174696F6E00005E202045D1
:101710006C65766174696F6E2063616C6962726179
:1017200074696F6E00002F20204F776E20636F6FFB
:101730007264696E617465202D206C6174697475C2
:10174000646500005C20204F776E20636F6F7264C9
:10175000696E617465202D206C6F6E6769747564A5
:10176000650061616120497320416E2056616C758E
:101770006520466F722054686520417A696D7574E2
:10178000682028302D33363029006565652049737F
:1017900020416E2056616C756520466F722054683A
:1017A0006520456C65766174696F6E2028302D3137
:1017B00038302900302E3500302E3100312E3000E7
:1017C000302E3200507265636973696F6E207365E5
:1017D0007420746F20005A65726F20706F73697483
:1017E000696F6E206F6E20004D6178696D756D2098
:1017F000656C65766174696F6E206973200042655F
:10180000657065723A2000004672657175656E6399
:1018100079004469726563742063757272656E74D1
:101820000000456C65766174696F6E2069732000F5
:101830004D6178696D756D206F6620617A696D758F
:1018400074683D20000056616C7565207361766593
:101850006400547970653A204753323332002D2D9D
:101860002D2D2D2D2D4C495354204F4620504152A3
:10187000414D45544552532D2D2D2D2D2D2D00001C
:101880004F6666736574206F6620617A696D757442
:10189000683A20004F6666736574206F6620656C39
:1018A00065766174696F6E3A20004D6178696D7577
:1018B0006D20706F736974696F6E206F6620617A36
:1018C000696D7574683A20004D6178696D756D2099
:1018D000706F736974696F6E206F6620656C6576D2
:1018E0006174696F6E3A20004D61782E20656C65D9
:1018F000766174696F6E20666F72206F76657274A0
:1019000075726E696E673A200000456C6576617489
:10191000696F6E20636F6E74726F6C3A2000506155
:10192000726B696E67206F6E20415A3A20005A65CB
:10193000726F20706F736974696F6E3A2000434F45
:101940004D20706F7274206563686F3A200044699F
:10195000726563742043757272656E740000507214
:1019600065636973696F6E3A20004C6174697475C0
:1019700064653A20000020204C6F6E6769747564BE
:10198000653A2000536F66747761726520766572E0
:1019900073696F6E3A20000041726520796F75207F
:1019A000737572653F00417A696D7574682069735B
:1019B0002063616C6962726174656400417A696D6B
:1019C0007574682063616C6962726174696E672006
:1019D0006572726F7200456C65766174696F6E2016
:1019E00069732063616C6962726174656400456C3F
:1019F00065766174696F6E2063616C69627261748F
:101A0000696E67206572726F7200466F726D6174E5
:101A10003A202F44442E44440000466F726D617496
:101A20003A205C4444442E444400454C3A204572DC
:101A3000726F7200415A3A204572726F7200444FC1
:101A4000574E2055502053544F5020434357202089
:101A500043570000415A494D5554483A2000415AD5
:101A6000494D5554483A204572726F72202020200B
:101A700020200000202020202020202053544F50E0
:101A800020434357202043570000202020202020BF
:101A900020204D454E5520202020202020200000D1
:101AA0002020202020202020202020202020202036
:101AB00020202020000053455420415A494D5554C0
:101AC0004820544F2020000053455420454C455693
:101AD00041542E20544F202000005041524B494E7B
:101AE0004720415A494D5554482000005041524B1F
:101AF0002E20454C45564154494F4E200000415A36
:101B0000494D555448204F46465345542020000027
:101B1000454C455641542E204F46465345542020AF
:101B200000004D4158494D554D20415A494D55549D
:101B3000482000004D415820454C202D204F56454F
:101B400052542E200000434F4D20504F52542045F8
:101B500043484F2049532000454C45564154494F76
:101B60004E20434F4E54522E2000434F4D4D554E64
:101B700049434154494F4E204753323332002020CD
:101B8000204120202020422000004D4158494D5541
:101B90004D20454C455641542E2000002020203930
:101BA00030202031383000005A45524F20504F49E4
:101BB0004E54204F4E2000004E4F52442020000033
:101BC000534F555448200000202020204E20202034
:101BD00053200000424545504552202020004F46EA
:101BE0004620202020202020200044697265637454
:101BF000204375722E004652455155454E4359209B
:101C0000200020204F4646202044432020465251A9
:101C100000002020202056657273696F6E2000003E
:101C2000505245434953494F4E202000302E312019
:101C3000646567202000302E322064656720200014
:101C4000302E3520646567202000312E30206465F9
:101C5000672020005345542041534C20544F2020EE
:101C600020004155544F205455524E494E47202094
:101C7000202020004F5645525455524E494E472081
:101C80002020202020004E4D454120544553542013
:101C9000202020202020200043414C494252415422
:101CA000494F4E2020415A4920454C4500002020F4
:101CB00020415A4920454C45000043414C4942527D
:101CC0004154494F4E20504C532057414954000035
:101CD0002020202020202020000020202020202044
:101CE0002000474741002020204F4B2020200000AB
:101CF0002020204F464620204F4E00003031323306
:101D00003435363738394142434445463031323331
:101D1000343536373839414243444546400E366EF5
:101D2000006ACF0EAF6EB06A240EAC6E900EAB6E32
:101D300000010F0EC16E070EB46E0301776B766B58
:101D4000756B7F0E746F0001896A8A6A8B6A8C6A70
:101D50008D6AC00E926E870E936EBE0E946ED00E7C
:101D6000956E880E966E310ECD6EB16A250E9D6E03
:101D7000A06A0B0EBD6EFA0EBF6EBE6ABA6AF40E92
:101D8000D36E400E9B6EC00EF26E700EF16EC00EE2
:101D9000F06E070EB46EC66AC26A0F0EC16EC06ADC
:101DA000900EAB6E200EAC6E080EB86EAC98AC8484
:101DB000030EB06E400EAF6E02EE02F0110EF76E23
:101DC000960EF66E9AEC02F0EF6A0301020E466F71
:101DD00093988A9893968A96939A8A9A939C8A9CC7
:101DE00095968C9695928C9295908C9094908B90E1
:101DF0003E983B9A3B9C416B426B406B3D983B98B5
:101E00003C9A236B226B216B206B276B266B256B17
:101E1000246B3C8E83AC3C9E3D8083AE3D903D84E4
:101E20003D823A9C3A9E3B923B900001A26BB36B81
:101E3000B26BB56BB46B0301640E4B6F00019F6B0B
:101E4000A06B010E8F6F05EC00F0110EF76EAC0E5B
:101E5000F66E2CEC01F0110EF76EC20EF66E2CEC45
:101E600001F0800E016E77C325F076C324F075C3B0
:101E700023F074C322F0010E98EC00F0640EBAEC6B
:101E800001F0FE0E34EC01F0400E34EC01F0000ED7
:101E900034EC01F0040E34EC01F0040E34EC01F0EB
:101EA000040E34EC01F0150E34EC01F00E0E34EC9F
:101EB00001F0040E34EC01F0000E34EC01F01E0EC3
:101EC000BAEC01F0FE0E34EC01F0480E34EC01F0F7
:101ED000000E34EC01F0040E34EC01F00E0E34EC84
:101EE00001F0150E34EC01F0040E34EC01F0040E98
:101EF00034EC01F0040E34EC01F0000E34EC01F08F
:101F00001E0EBAEC01F0FE0E34EC01F0500E34EC73
:101F100001F0000E34EC01F0040E34EC01F0020E7E
:101F200034EC01F01F0E34EC01F0020E34EC01F041
:101F3000040E34EC01F0000E34EC01F0000E34EC31
:101F400001F01E0EBAEC01F0FE0E34EC01F0580E5A
:101F500034EC01F0000E34EC01F0040E34EC01F02E
:101F6000080E34EC01F01F0E34EC01F0080E34ECD6
:101F700001F0040E34EC01F0000E34EC01F0000E20
:101F800034EC01F01E0EBAEC01F0FE0E34EC01F060
:101F9000600E34EC01F0000E34EC01F0010E34EC74
:101FA00001F0050E34EC01F0090E34EC01F01F0EC7
:101FB00034EC01F0080E34EC01F0040E34EC01F0C6
:101FC000000E34EC01F01E0EBAEC01F0FE0E34EC03
:101FD00001F0680E34EC01F0040E34EC01F00A0E4E
:101FE00034EC01F0040E34EC01F0000E34EC01F09E
:101FF000000E34EC01F0000E34EC01F0000E34EC75
:1020000001F0000E34EC01F01E0EBAEC01F0110EDE
:10201000F76ED40EF66E86EC01F0040E016E77C3F7
:1020200025F076C324F075C323F074C322F0010EAB
:1020300098EC00F00D0E8EEC01F00A0E8EEC01F023
:10204000AA6AA96AB3EC01F0436EB3EC01F0446EE6
:10205000AA6A020EA96EB3EC01F0456EB3EC01F072
:10206000466EAA6A040EA96EB3EC01F0646EB3EC7E
:1020700001F0656EAA6A060EA96EB3EC01F0666EF9
:10208000B3EC01F0676EAA6A080EA96EB3EC01F01A
:102090006C6EB3EC01F06D6EAA6A0A0EA96EB3EC19
:1020A00001F06E6EB3EC01F06F6EAA6A0C0EA96EB1
:1020B000B3EC01F0706EB3EC01F0716EAA6A0E0E13
:1020C000A96EB3EC01F0636EAA6A0F0EA96EB3ECB1
:1020D00001F0936FAA6A100EA96EB3EC01F0030130
:1020E000496FAA6A110EA96EB3EC01F00301456FA6
:1020F000AA6A120EA96EB3EC01F003012A6FB3ECC9
:1021000001F003012B6FB3EC01F003012C6FB3EC72
:1021100001F003012D6FAA6A160EA96EB3EC01F04F
:1021200003012E6FB3EC01F003012F6FB3EC01F04C
:102130000301306FB3EC01F00301316FAA6A1A0E8C
:10214000A96EB3EC01F00301326FB3EC01F00301AF
:10215000336F020E455DD8A4010E336E040E455D4B
:10216000D8A4010E33160A0E455DD8A4010E33160D
:10217000140E455DD8A4010E3316000103E00301DF
:10218000040E456F000144C050F043C04FF046C0FC
:1021900052F045C051F044C054F043C053F046C023
:1021A00056F045C055F003014551B40DF3CFBAF0D8
:1021B000F4CFBBF04551680DF3CFBCF0F4CFBDF0C8
:1021C0000001BD27635003014503F4CFBFF0F3CFF7
:1021D000BEF045510A0DF3CFC0F0F4CFC1F0455128
:1021E000640DF3CFC2F0F4CFC3F045511E0DF3CF11
:1021F000C6F0F4CFC7F04551320DF3CFC4F0F4CFA1
:10220000C5F045510F0DF3CFC8F0F4CFC9F03A94A3
:102210003A963A903A9246C042F045C041F00001E9
:102220009351E8BA01D0938EF088F28E04D0F2BEBA
:102230001200BBEF48F0FBDF070E146ED00EBBECB4
:1022400001F00001F4DFF3DF01EE37F0EF6AEFDFBA
:10225000EEDF00EEE6F0EF6AEADFE9DF3D98E7DF68
:1022600017EC48F0E4DF81A42AD0E1DF05EC00F0B0
:10227000DEDF93968A96DBDF93988A98D8DF939A6D
:102280008A9AD5DF939C8A9CD2DF95968C96CFDF75
:10229000CEDF3E98CCDFAA6AA96A4350A3EC01F0D6
:1022A0004450A3EC01F0C3DFAA6A020EA96E4550A8
:1022B000A3EC01F04650A3EC01F0B9DFFFD7B7DF84
:1022C000000E82B0010E336E3DBC3DAE02D0000E5A
:1022D00001D0010E331200013EB03EA202D0000E2A
:1022E00001D0010E3312000118E0A1DF010E80BC05
:1022F000000E336E010E80BE000E3312010E82B44A
:10230000000E3312010E82B6000E331206E08FDF8C
:102310008EDF3E988CDF95968C9689DFABA206D037
:1023200086DF85DFAB9883DF82DFAB8880DF010E3D
:1023300080BC000E336E000E3ABC010E331214E066
:1023400076DF75DF3A8C3AA43A9C71DF3AB80BD04D
:102350006EDF6DDF020E435C4F6E000E4458506E10
:1023600066DF65DF3A881AD062DF010E3AB8000EE8
:10237000336E000E3BB8010E331210E058DF010E31
:102380003AB4000E336E010E3AB0000E331606E07A
:102390004EDF93988A984BDF4ADF3E9848DF010E64
:1023A00080BE000E336E000E3ABE010E331214E0F2
:1023B0003EDF3DDF3A8E3AA43A9E39DF3AB80BD081
:1023C00036DF35DF020E43244F6E000E4420506E80
:1023D0002EDF2DDF3A881AD02ADF010E3AB8000E20
:1023E000336E000E3BB8010E331210E020DF010EF9
:1023F0003AB4000E336E010E3AB0000E331606E00A
:1024000016DF93968A9613DF12DF3E9810DF935102
:10241000E8B270D00CDF010E82B4000E336E000EF5
:102420003BB0010E331214E002DF01DF3B803AA61D
:102430003B90FDDE3ABA0BD0FADEF9DE020E4524FF
:10244000516E000E4620526EF2DEF1DE3A8A1AD04C
:10245000EEDE010E3ABA000E336E000E3BB8010EEE
:10246000331210E0E4DE010E3AB6000E336E010EB8
:102470003AB2000E331606E0DADE939A8A9AD7DE75
:10248000D6DE3E98D4DE010E82B6000E336E000E0C
:102490003BB2010E331214E0CADEC9DE3B823AA61B
:1024A0003B92C5DE3ABA0BD0C2DEC1DE020E455CFD
:1024B000516E000E4658526EBADEB9DE3A8A1AD014
:1024C000B6DE010E3ABA000E336E000E3BB8010EB6
:1024D000331210E0ACDE010E3AB6000E336E010E80
:1024E0003AB2000E331606E0A2DE939C8A9C9FDE71
:1024F0009EDE3E989CDE9BDE6C50435C476E6D50CA
:102500004458486E94DE48BE02D0000E01D0010E41
:10251000336E4750BC5D4850BD594850BD19D8B0C6
:10252000800A02E7000E01D0010E331204E07FDEC4
:102530007EDE838203D07BDE7ADE839278DE935167
:10254000E8A619D074DE73DEBA514726BB51482283
:102550006EDEBC51475CBD5148584850BD19D8B0DB
:10256000800A08E764DE63DEBC51475C476EBD51FC
:102570004858486E1BD05BDE48AE06D058DE57DEAA
:10258000BC514726BD51482252DEBC51475CBD516B
:1025900048584850BD19D8B0800A08E748DE47DEE1
:1025A000BC51475C476EBD514858486E40DE82B210
:1025B00003D03DDE8BEC2EF03ADE010E80BC000E27
:1025C000336E010E80BE000E33123BE030DE43500E
:1025D000535C0F6E44505458106E91EC02F0076E2D
:1025E00010C008F00750C85D0850C9590850C919F3
:1025F000D8B0800A0DE61BDE9351E8AC09D017DE97
:1026000016DE3A8414DE95968C8611DE10DE3E8846
:102610000EDE3DA215D00BDE0ADE3A9408DE07DEA0
:102620003A9805DE04DE3A9C02DE01DE3A9EFFDDCA
:10263000FEDD3D92FCDDFBDD44C054F043C053F0B1
:1026400006D0F5DDF4DD44C054F043C053F0EFDDB7
:10265000010E82B6000E336E010E82B4000E3312EC
:102660004FE017EC11F04550555C0F6E4650565830
:10267000106E91EC02F0076E10C008F00750C05DBC
:102680000850C1590850C119D8B0800A13E617EC98
:1026900011F09351E8AC0ED017EC11F017EC11F0DB
:1026A0003A8617EC11F095968C8617EC11F017EC22
:1026B00011F03E8817EC11F03DA421D017EC11F079
:1026C00017EC11F03A9617EC11F017EC11F03A9A5A
:1026D00017EC11F017EC11F03B9217EC11F017EC1E
:1026E00011F03B9017EC11F017EC11F03D9417EC42
:1026F00011F017EC11F046C056F045C055F008D067
:1027000017EC11F017EC11F046C056F045C055F02B
:1027100017EC11F0010E80BC000E336E010E80BE6E
:10272000000E3312010E82B6000E3312010E82B477
:10273000000E3312D8B46CD017EC11F03BA868D05F
:1027400017EC11F0E86A80BC010F80BE010F086A27
:10275000076E085203E1020E075C02E3000E01D08F
:10276000010E336E000E3DB2010E331600011CE067
:1027700017EC11F093968A9617EC11F093988A98BB
:1027800017EC11F0010E81BA000E336E010E81BC00
:10279000000E331609E017EC11F095968C9617ECA5
:1027A00011F017EC11F03E9817EC11F0E86A82B4C2
:1027B000010F82B6010F086A076E085203E1020E8C
:1027C000075C02E3000E01D0010E336E000E3DB433
:1027D000010E331600011CE017EC11F0939A8A9A4F
:1027E00017EC11F0939C8A9C17EC11F0010E81B646
:1027F000000E336E010E81B8000E331609E017EC9F
:1028000011F095968C9617EC11F017EC11F03E989C
:1028100017EC11F03AA682D017EC11F06E50455C1F
:10282000076E6F504658086E08BE05D00750081056
:1028300002E0000E01D0010E336E000E81BC010ECD
:10284000331621E017EC11F017EC11F03A9617EC63
:1028500011F017EC11F03A9A17EC11F017EC11F097
:102860003B9217EC11F017EC11F03D9417EC11F0BE
:10287000939C8A9C17EC11F095968C9617EC11F0AE
:1028800017EC11F03E9817EC11F06E50455C076E96
:102890006F504658086E0750BE5D0850BF5908502B
:1028A000BF19D8B0800A02E7000E01D0010E336EC6
:1028B000000E81BA010E331621E017EC11F017EC6F
:1028C00011F03A9617EC11F017EC11F03A9A17EC58
:1028D00011F017EC11F03B9017EC11F017EC11F020
:1028E0003D9417EC11F0939A8A9A17EC11F0959693
:1028F0008C9617EC11F017EC11F03E9817EC11F0D4
:10290000000E82B4010E336E000E82B6010E331635
:1029100005E017EC11F017EC11F03D8417EC11F005
:102920003AA482D017EC11F06C50435C076E6D50E6
:102930004458086E08BE05D00750081002E0000E8B
:1029400001D0010E336E000E81B8010E331621E066
:1029500017EC11F017EC11F03A9417EC11F017EC9A
:1029600011F03A9817EC11F017EC11F03A9C17ECB3
:1029700011F017EC11F03D9217EC11F093988A9832
:1029800017EC11F095968C9617EC11F017EC11F0EE
:102990003E9817EC11F06C50435C076E6D50445834
:1029A000086EBC51075CBD5108580850BD19D8B01D
:1029B000800A02E6000E01D0010E336E000E81B6D1
:1029C000010E331621E017EC11F017EC11F03A94D8
:1029D00017EC11F017EC11F03A9817EC11F017EC16
:1029E00011F03A9E17EC11F017EC11F03D9217EC34
:1029F00011F093968A9617EC11F095968C9617EC39
:102A000011F017EC11F03E9817EC11F0000E80BC9D
:102A1000010E336E000E80BE010E331605E017EC7A
:102A200011F017EC11F03D8217EC11F03AA889D0A3
:102A300017EC11F043504F5C44505058445050181C
:102A4000D8B0800A1FE617EC11F081A608D017EC69
:102A500011F093968A9617EC11F0D0EC3DF017EC3C
:102A600011F017EC11F03D9C17EC11F017EC11F080
:102A70003D8E17EC11F093988A8817EC11F017EC43
:102A800011F03E8817EC11F04F50435C5050445801
:102A900044505018D8B0800A1FE617EC11F081A8F6
:102AA00008D017EC11F093988A9817EC11F0D0EC3D
:102AB0003DF017EC11F017EC11F03D9E17EC11F002
:102AC00017EC11F03D8C17EC11F093968A8617ECF9
:102AD00011F017EC11F03E8817EC11F05050445CE7
:102AE00030E14F50435C2DE117EC11F0000E80BE39
:102AF000010E336E010E3ABE000E331604E017ECE1
:102B000011F093968A9617EC11F0000E80BC010E1E
:102B1000336E010E3ABC000E331604E017EC11F0D0
:102B200093988A9817EC11F017EC11F03A9817EC7B
:102B300011F017EC11F03A9017EC11F017EC11F0BE
:102B40003E9817EC11F09351E8B292D017EC11F0C7
:102B50003BBC8DD017EC11F03AAA89D017EC11F0DC
:102B60004550515C4650525846505218D8B0800AD1
:102B70001FE617EC11F081AA08D017EC11F0939A18
:102B80008A9A17EC11F0D0EC3DF017EC11F017EC2D
:102B900011F03E9017EC11F017EC11F03E8217EC9B
:102BA00011F0939C8A8C17EC11F017EC11F03E8811
:102BB00017EC11F05150455C52504658465052188F
:102BC000D8B0800A1FE617EC11F081AC08D017ECE2
:102BD00011F0939C8A9C17EC11F0D0EC3DF017ECAF
:102BE00011F017EC11F03E9217EC11F017EC11F008
:102BF0003E8017EC11F0939A8A8A17EC11F017ECCB
:102C000011F03E8817EC11F05250465C30E1515003
:102C1000455C2DE117EC11F0000E82B6010E336E0B
:102C2000010E3BB2000E331604E017EC11F0939C3A
:102C30008A9C17EC11F0000E82B4010E336E010E67
:102C40003BB0000E331604E017EC11F0939A8A9A09
:102C500017EC11F017EC11F03A9A17EC11F017EC91
:102C600011F03A9217EC11F017EC11F03E9805D0E4
:102C700017EC11F017EC11F03A9A17EC11F0000E66
:102C80003AB4010E336E000E3AB6010E331209E06B
:102C900017EC11F095968C8617EC11F017EC11F0EB
:102CA0003E8817EC11F017EC11F06E50455C496E40
:102CB0006F5046584A6E17EC11F04ABE02D0000E13
:102CC00001D0010E336E4950BE5D4A50BF594A5083
:102CD000BF19D8B0800A02E7000E01D0010E3312EE
:102CE00006E017EC11F017EC11F0838005D017EC1B
:102CF00011F017EC11F0839017EC11F017EC11F0B4
:102D00003BB882803BA8829017EC11F012EC2AF0BD
:102D100017EC11F0000E82B6010E336E000E82B475
:102D2000010E331608E017EC11F017EC11F046C055
:102D300056F045C055F017EC11F0000E80BC010EA6
:102D4000336E000E80BE010E331608E017EC11F052
:102D500017EC11F044C054F043C053F017EC11F0DD
:102D6000000E3DB8010E336E000E3BB8010E331657
:102D700022E017EC11F0A3531EE017EC11F0106ADB
:102D8000A3C00FF0146A460E136EFDEC01F018C0DC
:102D900008F017C007F00850071004E117EC11F015
:102DA000CBEC47F017EC11F0A30717EC11F0010E74
:102DB000BAEC01F0E0D717EC11F03DA8C7EF28F00E
:102DC00017EC11F017EC11F03D9817EC11F0B50E5F
:102DD0000301735D000104E317EC11F09DEC50F06A
:102DE00017EC11F017EC11F00301736B17EC11F0F5
:102DF00017EC11F00001E651A96F17EC11F0240E49
:102E0000A95D06E117EC11F0FFEC3DF0C0EF28F0F2
:102E100017EC11F0570EA95DD8A499D017EC11F05A
:102E2000EA51076E200E075CD8A48FD017EC11F082
:102E300017EC11F001EE88F010EEE6F0060EF36EDE
:102E4000030EA9EC02F0EF6A17EC11F017EC11F089
:102E500003EE85F011EE88F0060EA2EC02F0DBEC3A
:102E600052F083C3ABF082C3AAF017EC11F0AB5160
:102E7000E8AE02D0000E01D0010E336EAB51E8BEB9
:102E800007D0AB5303E1AA51B40802E2000E01D00F
:102E9000010E33160001D8B458D017EC11F017EC1E
:102EA00011F0ABC07DF3AAC07CF39EEC52F07FC35F
:102EB00042F07EC341F017EC11F017EC11F001EE77
:102EC00088F010EEE6F0020EF36E030EA9EC02F0AD
:102ED000EF6A17EC11F017EC11F003EE85F011EE2C
:102EE00088F0060EA2EC02F0DBEC52F083C3ABF0EC
:102EF00082C3AAF017EC11F0AB51E8AE02D0000E7D
:102F000001D0010E336EAB51E8BE09D0010EAB5DAE
:102F100006E303E1690EAA5D02E3000E01D0010E93
:102F20003316000112E017EC11F017EC11F0ABC0F2
:102F300079F3AAC078F34BEC52F07BC340F07AC32C
:102F40003FF017EC11F0CBEC47F0C0EF28F04D0E3E
:102F5000A95DD8A4ACD017EC11F0E751076E520E62
:102F6000075C14E117EC11F017EC11F03A9017EC34
:102F700011F017EC11F03A8417EC11F017EC11F086
:102F80003A8E17EC11F0CBEC47F08FD04C0E075C6B
:102F900014E117EC11F017EC11F03A9017EC11F066
:102FA00017EC11F03A8417EC11F017EC11F03A8C91
:102FB00017EC11F0CBEC47F078D0550E075C14E11C
:102FC00017EC11F017EC11F03A9217EC11F017EC26
:102FD00011F03A8617EC11F017EC11F03B8017EC6A
:102FE00011F0CBEC47F061D0440E075C14E117EC14
:102FF00011F017EC11F03A9217EC11F017EC11F0F8
:103000003A8617EC11F017EC11F03B8217EC11F037
:10301000CBEC47F04AD017EC11F017EC11F001EEB1
:1030200088F010EEE6F0020EF36E030EA9EC02F04B
:10303000EF6A17EC11F017EC11F003EE85F011EECA
:1030400088F0060EA2EC02F0DBEC52F083C3ABF08A
:1030500082C3AAF017EC11F0AB51E8AE02D0000E1B
:1030600001D0010E336EAB51E8BE09D0010EAB5D4D
:1030700006E303E1690EAA5D02E3000E01D0010E32
:103080003316000112E017EC11F017EC11F0ABC091
:1030900079F3AAC078F34BEC52F07BC340F07AC3CB
:1030A0003FF017EC11F0CBEC47F0C0EF28F04B0EDF
:1030B000A95DD8A44AD017EC11F017EC11F001EE7D
:1030C00088F010EEE6F0020EF36E030EA9EC02F0AB
:1030D000EF6A17EC11F017EC11F003EE85F011EE2A
:1030E00088F0060EA2EC02F0DBEC52F083C3ABF0EA
:1030F00082C3AAF017EC11F0AB51E8AE02D0000E7B
:1031000001D0010E336EAB51E8BE07D0AB5303E1E3
:10311000AA51B40802E2000E01D0010E33160001DC
:1031200012E017EC11F017EC11F0ABC07DF3AAC060
:103130007CF39EEC52F07FC342F07EC341F017EC6B
:1031400011F0CBEC47F0C0EF28F0520EA95D15E16D
:1031500017EC11F017EC11F03A9017EC11F017EC96
:1031600011F03A8417EC11F017EC11F03A8E17ECCD
:1031700011F0CBEC47F0C0EF28F04C0EA95D15E143
:1031800017EC11F017EC11F03A9017EC11F017EC66
:1031900011F03A8417EC11F017EC11F03A8C17EC9F
:1031A00011F0CBEC47F0C0EF28F0550EA95D15E10A
:1031B00017EC11F017EC11F03A9217EC11F017EC34
:1031C00011F03A8617EC11F017EC11F03B8017EC78
:1031D00011F0CBEC47F0C0EF28F0440EA95D15E1EB
:1031E00017EC11F017EC11F03A9217EC11F017EC04
:1031F00011F03A8617EC11F017EC11F03B8217EC46
:1032000011F0CBEC47F0C0EF28F0530EA95DD8A425
:103210005ED017EC11F0E751076E410E075C15E127
:1032200017EC11F017EC11F03A9017EC11F017ECC5
:1032300011F03A9417EC11F017EC11F03A9C17ECDE
:1032400011F017EC11F03A9E40D0450E075C15E1E5
:1032500017EC11F017EC11F03A9217EC11F017EC93
:1032600011F03A9617EC11F017EC11F03B9017ECB7
:1032700011F017EC11F03B9228D017EC11F017EC7D
:1032800011F03A9017EC11F017EC11F03A9217EC9C
:1032900011F017EC11F03A9417EC11F017EC11F053
:1032A0003A9617EC11F017EC11F03A9C17EC11F06C
:1032B00017EC11F03A9E17EC11F017EC11F03B905F
:1032C00017EC11F017EC11F03B92C0EF28F0410E13
:1032D000A95DD8A4C8D017EC11F0E751076E5A0EBB
:1032E000075CD8A4AAD017EC11F017EC11F001EE8E
:1032F00088F010EEE6F0030EF36EA9EC02F0EF6A30
:1033000017EC11F017EC11F003EE85F011EE88F0D8
:10331000060EA2EC02F0DBEC52F083C3ABF082C3EA
:10332000AAF017EC11F0AB51E8AE02D0000E01D0BC
:10333000010E336EAB51E8BE09D0010EAB5D06E362
:1033400003E1690EAA5D02E3000E01D0010E3316FF
:103350000001D8B471D017EC11F017EC11F0ABC02C
:1033600079F3AAC078F34BEC52F07BC340F07AC3F8
:103370003FF017EC11F0ED51076E200E075C010EC7
:10338000D8A4000E336EEE51076E450E075C010E99
:10339000D8A4000E3316EF51076E4C0E075C010ED9
:1033A000D8A4000E331644E017EC11F017EC11F01E
:1033B00001EE88F010EEE6F00B0EF36E030EA9ECB2
:1033C00002F0EF6A17EC11F017EC11F003EE85F044
:1033D00011EE88F0060EA2EC02F0DBEC52F083C393
:1033E000ABF082C3AAF017EC11F0AB51E8AE02D0FB
:1033F000000E01D0010E336EAB51E8BE07D0AB53C7
:1034000003E1AA51B40802E2000E01D0010E331606
:1034100000010EE017EC11F017EC11F0ABC07DF3DA
:10342000AAC07CF39EEC52F07FC342F07EC341F011
:1034300017EC11F0CBEC47F014D017EC11F017ECAF
:1034400011F03A9017EC11F017EC11F03A9417ECD8
:1034500011F017EC11F03A9C17EC11F017EC11F089
:103460003A9EC0EF28F0450EA95DD8A465D017ECB0
:1034700011F0E751076E4C0E075C48E117EC11F0B4
:1034800017EC11F001EE88F010EEE6F0030EF36E8B
:10349000A9EC02F0EF6A17EC11F017EC11F003EE53
:1034A00085F011EE88F0060EA2EC02F0DBEC52F093
:1034B00083C3ABF082C3AAF017EC11F0AB51E8AEB6
:1034C00002D0000E01D0010E336EAB51E8BE07D022
:1034D000AB5303E1AA51B40802E2000E01D0010E81
:1034E0003316000112E017EC11F017EC11F0ABC02D
:1034F0007DF3AAC07CF39EEC52F07FC342F07EC302
:1035000041F017EC11F0CBEC47F014D017EC11F0B0
:1035100017EC11F03A9217EC11F017EC11F03A9603
:1035200017EC11F017EC11F03B9017EC11F017ECC1
:1035300011F03B92C0EF28F0430EA95DD8A4CCD087
:1035400017EC11F0E751076E320E075CD8A479D062
:1035500017EC11F09351E8B437D017EC11F02B0EA3
:103560008EEC01F0300E8EEC01F0040E016E030EB5
:10357000056E48C01EF047C01DF045C317F0186A1D
:1035800014EC02F0176E10C018F060EC00F02B0E77
:103590008EEC01F0300E8EEC01F0030E056E4AC089
:1035A0001EF049C01DF045C317F0186A14EC02F074
:1035B000176E10C018F060EC00F00D0E8EEC01F0EC
:1035C0000A0E8EEC01F03CD017EC11F0410E8EEC9F
:1035D00001F05A0E8EEC01F03D0E8EEC01F0040E5F
:1035E000016E030E056E48C01EF047C01DF045C3B6
:1035F00017F0186A14EC02F0176E10C018F060ECA7
:1036000000F0450E8EEC01F04C0E8EEC01F03D0EFC
:103610008EEC01F0030E056E4AC01EF049C01DF08D
:1036200045C317F0186A14EC02F0176E10C018F0BA
:1036300060EC00F00D0E8EEC01F00A0E8EEC01F045
:1036400049D017EC11F09351E8B421D017EC11F0E8
:103650002B0E8EEC01F0300E8EEC01F0040E016E9C
:10366000030E056E48C01EF047C01DF045C317F09D
:10367000186A14EC02F0176E10C018F060EC00F03D
:103680000D0E8EEC01F00A0E8EEC01F023D017EC3B
:1036900011F0410E8EEC01F05A0E8EEC01F03D0E51
:1036A0008EEC01F0040E016E030E056E48C01EF094
:1036B00047C01DF045C317F0186A14EC02F0176EEE
:1036C00010C018F060EC00F00D0E8EEC01F00A0E48
:1036D0008EEC01F0C0EF28F0420EA95D4BE117EC33
:1036E00011F09351E8B421D017EC11F02B0E8EECB1
:1036F00001F0300E8EEC01F0040E016E030E056E2B
:103700004AC01EF049C01DF045C317F0186A14ECFA
:1037100002F0176E10C018F060EC00F00D0E8EEC89
:1037200001F00A0E8EEC01F023D017EC11F0450EDB
:103730008EEC01F04C0E8EEC01F03D0E8EEC01F0A3
:10374000040E016E030E056E4AC01EF049C01DF046
:1037500045C317F0186A14EC02F0176E10C018F089
:1037600060EC00F00D0E8EEC01F00A0E8EEC01F014
:10377000C0EF28F0560EA95D40E117EC11F0E751BB
:10378000076E450E075C1CE117EC11F0560E8EEC2F
:1037900001F0450E8EEC01F0040E016E77C325F0AA
:1037A00076C324F075C323F074C322F0010E98ECA5
:1037B00000F00D0E8EEC01F00A0E8EEC01F01BD025
:1037C00017EC11F0110EF76EF20EF66E86EC01F0AA
:1037D000040E016E77C325F076C324F075C323F081
:1037E00074C322F0010E98EC00F00D0E8EEC01F087
:1037F0000A0E8EEC01F0C0EF28F0500EA95DD8A49F
:103800004ED117EC11F0E751076E3F0E075C3DE11A
:1038100017EC11F0110EF76EFC0EF66E86EC01F04F
:10382000040E016E030E056E65C01EF064C01DF02F
:1038300045C317F0186A14EC02F0176E10C018F0A8
:1038400060EC00F0200E8EEC01F0450E8EEC01F0E5
:103850004C0E8EEC01F03D0E8EEC01F0030E056E69
:1038600067C01EF066C01DF045C317F0186A14EC5F
:1038700002F0176E10C018F060EC00F00D0E8EEC28
:1038800001F00A0E8EEC01F008D117EC11F0E751AF
:10389000076E210E075C27E117EC11F017EC11F011
:1038A00044C065F043C064F017EC11F017EC11F060
:1038B00046C067F045C066F017EC11F0AA6A040E26
:1038C000A96E6450A3EC01F06550A3EC01F017EC75
:1038D00011F0AA6A060EA96E6650A3EC01F06750BB
:1038E000A3EC01F0DAD017EC11F0E751076E300EBF
:1038F000075C000ED8B0010E336EE751076E3A0E2A
:10390000075C02E3000E01D0010E3316D8B4ABD031
:1039100017EC11F017EC11F001EE88F010EEE6F064
:10392000020EF36E030EA9EC02F0EF6A17EC11F031
:1039300017EC11F003EE85F011EE88F0060EA2EC04
:1039400002F0DBEC52F083C3ABF082C3AAF017ECB9
:1039500011F0AB51E8BE09D0010EAB5D06E303E107
:10396000690EAA5D02E3000E01D0010E336E000164
:10397000AB51E8AE02D0000E01D0010E331616E0B6
:1039800017EC11F017EC11F0AA5103014503F3CF26
:1039900064F0F4CF65F00001AB5103014503F3502F
:1039A000652645AF03D00001AA51655E000117EC02
:1039B00011F017EC11F001EE88F010EEE6F0060EB3
:1039C000F36E030EA9EC02F0EF6A17EC11F017EC9E
:1039D00011F003EE85F011EE88F0060EA2EC02F075
:1039E000DBEC52F083C3ABF082C3AAF017EC11F00A
:1039F000AB51E8BE37D017EC11F0ABBF05D0AB51DF
:103A00001AE1B50EAA5D17E217EC11F017EC11F0F0
:103A10000001AA5103014503F3CF66F0F4CF67F02C
:103A20000001AB5103014503F350672645AF03D0B6
:103A30000001AA51675E000117EC11F0AA6A040E9A
:103A4000A96E6450A3EC01F06550A3EC01F017ECF3
:103A500011F0AA6A060EA96E6650A3EC01F0675039
:103A6000A3EC01F01AD017EC11F017EC11F065C0BF
:103A700040F064C03FF017EC11F017EC11F067C094
:103A800042F066C041F017EC11F017EC11F03A80EB
:103A900017EC11F017EC11F03A82C0EF28F04F0E3E
:103AA000A95DD8A4B0D017EC11F0E751076E3F0E16
:103AB000075C20E117EC11F0120EF76E080EF66E9F
:103AC00086EC01F0040E016E056A6DC01EF06CC03C
:103AD0001DF045C317F0186A14EC02F0176E10C001
:103AE00018F060EC00F00D0E8EEC01F00A0E8EEC7A
:103AF00001F087D017EC11F0E751076E210E075C3B
:103B00001AE117EC11F0AA6A080EA96E4350A3EC53
:103B100001F04450A3EC01F017EC11F0120EF76E17
:103B20001A0EF66E86EC01F00D0E8EEC01F00A0E08
:103B30008EEC01F066D017EC11F017EC11F001EEED
:103B400088F010EEE6F0020EF36E030EA9EC02F020
:103B5000EF6A17EC11F017EC11F003EE85F011EE9F
:103B600088F0060EA2EC02F0DBEC52F083C3ABF05F
:103B700082C3AAF017EC11F0AB51E8AE02D0000EF0
:103B800001D0010E336EAB51E8BE07D0AB5303E159
:103B9000AA51320802E2000E01D0010E33160001D4
:103BA0002FE017EC11F017EC11F0AA5103014503B7
:103BB000F3CF6CF0F4CF6DF00001AB51030145037E
:103BC000F3506D2645AF03D00001AA516D5E17EC8E
:103BD00011F0AA6A080EA96E6C50A3EC01F06D50AA
:103BE000A3EC01F017EC11F0120EF76E1A0EF66E40
:103BF00086EC01F00D0E8EEC01F00A0E8EEC01F059
:103C00000001C0EF28F0470EA95DD8A48FD017ECB3
:103C100011F0E751076E3F0E075C20E117EC11F041
:103C2000120EF76E300EF66E86EC01F0040E016E89
:103C3000056A6FC01EF06EC01DF045C317F0186A0C
:103C400014EC02F0176E10C018F060EC00F00D0ECE
:103C50008EEC01F00A0E8EEC01F066D017EC11F03C
:103C600017EC11F001EE88F010EEE6F0020EF36EA4
:103C7000030EA9EC02F0EF6A17EC11F017EC11F04B
:103C800003EE85F011EE88F0060EA2EC02F0DBECFC
:103C900052F083C3ABF082C3AAF017EC11F0AB5122
:103CA000E8AE02D0000E01D0010E336EAB51E8BE7B
:103CB00007D0AB5303E1AA511E0802E2000E01D067
:103CC000010E331600012FE017EC11F017EC11F084
:103CD000AA5103014503F3CF6EF0F4CF6FF000015A
:103CE000AB5103014503F3506F2645AF03D00001EC
:103CF000AA516F5E17EC11F0AA6A0A0EA96E6E50F7
:103D0000A3EC01F06F50A3EC01F017EC11F0120ED0
:103D1000F76E440EF66E86EC01F00D0E8EEC01F09F
:103D20000A0E8EEC01F00001C0EF28F0480EA95DEC
:103D300004E03F0EA95DD8A478D217EC11F0120E62
:103D4000F76E5C0EF66E86EC01F00D0E8EEC01F057
:103D50000A0E8EEC01F017EC11F0120EF76E860EC3
:103D6000F66E86EC01F00D0E8EEC01F00A0E8EEC74
:103D700001F017EC11F0120EF76E940EF66E86EC51
:103D800001F00D0E8EEC01F00A0E8EEC01F017EC36
:103D900011F0120EF76EAC0EF66E86EC01F00D0E01
:103DA0008EEC01F00A0E8EEC01F017EC11F0120E01
:103DB000F76EC40EF66E86EC01F00D0E8EEC01F07F
:103DC0000A0E8EEC01F017EC11F0120EF76EDC0EFD
:103DD000F66E86EC01F00D0E8EEC01F00A0E8EEC04
:103DE00001F017EC11F0120EF76EF80EF66E86EC7D
:103DF00001F00D0E8EEC01F00A0E8EEC01F017ECC6
:103E000011F0130EF76E140EF66E86EC01F00D0E27
:103E10008EEC01F00A0E8EEC01F017EC11F0130E8F
:103E2000F76E380EF66E86EC01F00D0E8EEC01F09A
:103E30000A0E8EEC01F017EC11F0130EF76E620E05
:103E4000F66E86EC01F00D0E8EEC01F00A0E8EEC93
:103E500001F017EC11F0130EF76E900EF66E86EC73
:103E600001F00D0E8EEC01F00A0E8EEC01F017EC55
:103E700011F0130EF76EB40EF66E86EC01F00D0E17
:103E80008EEC01F00A0E8EEC01F017EC11F0130E1F
:103E9000F76ECE0EF66E86EC01F00D0E8EEC01F094
:103EA0000A0E8EEC01F017EC11F0130EF76EEE0E09
:103EB000F66E86EC01F00D0E8EEC01F00A0E8EEC23
:103EC00001F017EC11F0130EF76EFC0EF66E86EC97
:103ED00001F00D0E8EEC01F00A0E8EEC01F017ECE5
:103EE00011F0140EF76E100EF66E86EC01F00D0E4A
:103EF0008EEC01F00A0E8EEC01F017EC11F0140EAE
:103F0000F76E320EF66E86EC01F00D0E8EEC01F0BF
:103F10000A0E8EEC01F017EC11F0140EF76E500E35
:103F2000F66E86EC01F00D0E8EEC01F00A0E8EECB2
:103F300001F017EC11F0140EF76E620EF66E86ECBF
:103F400001F00D0E8EEC01F00A0E8EEC01F017EC74
:103F500011F0140EF76E8C0EF66E86EC01F00D0E5D
:103F60008EEC01F00A0E8EEC01F017EC11F0140E3D
:103F7000F76EAA0EF66E86EC01F00D0E8EEC01F0D7
:103F80000A0E8EEC01F017EC11F0140EF76ED40E41
:103F9000F66E86EC01F00D0E8EEC01F00A0E8EEC42
:103FA00001F017EC11F0140EF76EE40EF66E86ECCD
:103FB00001F00D0E8EEC01F00A0E8EEC01F017EC04
:103FC00011F0140EF76EFC0EF66E86EC01F00D0E7D
:103FD0008EEC01F00A0E8EEC01F017EC11F0150ECC
:103FE000F76E260EF66E86EC01F00D0E8EEC01F0EB
:103FF0000A0E8EEC01F017EC11F0150EF76E3E0E66
:10400000F66E86EC01F00D0E8EEC01F00A0E8EECD1
:1040100001F017EC11F0150EF76E6A0EF66E86ECD5
:1040200001F00D0E8EEC01F00A0E8EEC01F017EC93
:1040300011F0150EF76E880EF66E86EC01F00D0E7F
:104040008EEC01F00A0E8EEC01F017EC11F0150E5B
:10405000F76EAA0EF66E86EC01F00D0E8EEC01F0F6
:104060000A0E8EEC01F017EC11F0150EF76EC00E73
:10407000F66E86EC01F00D0E8EEC01F00A0E8EEC61
:1040800001F017EC11F0150EF76ECC0EF66E86EC03
:1040900001F00D0E8EEC01F00A0E8EEC01F017EC23
:1040A00011F0150EF76EE60EF66E86EC01F00D0EB1
:1040B0008EEC01F00A0E8EEC01F017EC11F0150EEB
:1040C000F76EFA0EF66E86EC01F00D0E8EEC01F036
:1040D0000A0E8EEC01F017EC11F0160EF76E220EA0
:1040E000F66E86EC01F00D0E8EEC01F00A0E8EECF1
:1040F00001F017EC11F0160EF76E340EF66E86EC2A
:1041000001F00D0E8EEC01F00A0E8EEC01F017ECB2
:1041100011F0160EF76E5C0EF66E86EC01F00D0EC9
:104120008EEC01F00A0E8EEC01F017EC11F0160E79
:10413000F76E940EF66E86EC01F00D0E8EEC01F02B
:104140000A0E8EEC01F017EC11F0160EF76EB20E9F
:10415000F66E86EC01F00D0E8EEC01F00A0E8EEC80
:1041600001F017EC11F0160EF76ED40EF66E86EC19
:1041700001F00D0E8EEC01F00A0E8EEC01F017EC42
:1041800011F0160EF76EF40EF66E86EC01F00D0EC1
:104190008EEC01F00A0E8EEC01F017EC11F0170E08
:1041A000F76E0C0EF66E86EC01F00D0E8EEC01F043
:1041B0000A0E8EEC01F017EC11F0170EF76E260EBA
:1041C000F66E86EC01F00D0E8EEC01F00A0E8EEC10
:1041D00001F017EC11F0170EF76E440EF66E86EC38
:1041E00001F00D0E8EEC01F00A0E8EEC01F017ECD2
:1041F00011F0170EF76E620EF66E86EC01F00D0EE2
:104200008EEC01F00A0E8EEC01F017EC11F0170E97
:10421000F76E8A0EF66E86EC01F00D0E8EEC01F054
:104220000A0E8EEC01F0C0EF28F0590EA95D4AE1AC
:1042300017EC11F017EC11F0000E93B1010E010A0A
:10424000D8B49391D8A4938117EC11F0450E8EEC5D
:1042500001F0630E8EEC01F0680E8EEC01F06F0E33
:104260008EEC01F0200E8EEC01F017EC11F0933182
:104270000FE317EC11F04F0E8EEC01F04E0E8EECAA
:1042800001F00D0E8EEC01F00A0E8EEC01F010D054
:1042900017EC11F04F0E8EEC01F0460E8EEC01F093
:1042A0008EEC01F00D0E8EEC01F00A0E8EEC01F09A
:1042B00017EC11F0AA6A0F0EA96E9351A3EC01F04E
:1042C000C0EF28F0510EA95DD8A4D9D017EC11F099
:1042D00017EC11F001EE88F010EEE6F0020EF36E2E
:1042E000030EA9EC02F0EF6A17EC11F0170EF76E4F
:1042F000B40EF66E01EE88F0BDEC02F012E117ECA0
:1043000011F017EC11F00301040E456F17EC11F0DA
:10431000AA6A110EA96E03014551A3EC01F0000138
:1043200065D017EC11F0170EF76EB80EF66E01EEB1
:1043300088F0BDEC02F012E117EC11F017EC11F06F
:104340000301140E456F17EC11F0AA6A110EA96E45
:1043500003014551A3EC01F0000148D017EC11F026
:1043600001EE88F0EECFF3FFEFCFF4FFF350310A08
:10437000F41002E0000E01D0010E336E170EF76E3E
:10438000BC0EF66E01EE88F0C6EC02F0331212E0BD
:1043900017EC11F017EC11F00301020E456F17EC4A
:1043A00011F0AA6A110EA96E03014551A3EC01F0A8
:1043B00000011CD017EC11F0170EF76EC00EF66E50
:1043C00001EE88F0BDEC02F010E117EC11F017ECF3
:1043D00011F003010A0E456F17EC11F0AA6A110ED5
:1043E000A96E03014551A3EC01F0000117EC11F097
:1043F00017EC11F0030145518AEC08F02DC031F0A3
:104400002CC030F02BC02FF02AC02EF02D6A2C6A61
:104410002B6A800E2A6E7DEC07F02DC0A7F02CC011
:10442000A6F02BC0A5F02AC0A4F017EC11F0170ECF
:10443000F76EC40EF66E86EC01F0040E016EA7C096
:1044400025F0A6C024F0A5C023F0A4C022F0010EE0
:1044500098EC00F0200E8EEC01F0640E8EEC01F072
:10446000650E8EEC01F0670E8EEC01F00D0E8EECF9
:1044700001F00A0E8EEC01F00001C0EF28F05A0E98
:10448000A95D4FE117EC11F017EC11F0000E93B796
:10449000010E010AD8B49397D8A4938717EC11F0B2
:1044A000170EF76ED60EF66E86EC01F017EC11F0D3
:1044B0009351E8A618D017EC11F0730E8EEC01F0B2
:1044C0006F0E8EEC01F0750E8EEC01F0740E8EEC1A
:1044D00001F0680E8EEC01F00D0E8EEC01F00A0E6C
:1044E0008EEC01F014D017EC11F06E0E8EEC01F092
:1044F0006F0E8EEC01F0720E8EEC01F0640E8EECFD
:1045000001F00D0E8EEC01F00A0E8EEC01F017ECAE
:1045100011F0AA6A0F0EA96E9351A3EC01F0C0EF3F
:1045200028F0260EA95D31E117EC11F05A0E635CFC
:1045300007E117EC11F017EC11F0B40E636E06D022
:1045400017EC11F017EC11F05A0E636E17EC11F026
:10455000170EF76EE80EF66E86EC01F0040E016E93
:10456000030E056E63505EEC00F00D0E8EEC01F054
:104570000A0E8EEC01F017EC11F0AA6A0E0EA96E6D
:104580006350A3EC01F0C0EF28F04A0EA95DD8A457
:1045900062D017EC11F0170EF76EFE0EF66E86EC79
:1045A00001F017EC11F0E751076E4E0E075C0FE1BA
:1045B00017EC11F06F0E8EEC01F0660E8EEC01F030
:1045C0008EEC01F017EC11F017EC11F0939B17EC47
:1045D00011F0E751076E460E075C12E117EC11F07F
:1045E000180EF76E080EF66E86EC01F017EC11F05F
:1045F00017EC11F0938917EC11F017EC11F0938B75
:1046000017EC11F0E751076E440E075C12E117EC4E
:1046100011F0180EF76E120EF66E86EC01F017EC24
:1046200011F017EC11F0939917EC11F017EC11F051
:10463000938B17EC11F00D0E8EEC01F00A0E8EEC40
:1046400001F017EC11F0AA6A0F0EA96E9351A3ECBA
:1046500001F0C0EF28F0250EA95D48E117EC11F03C
:1046600017EC11F0000E93B3010E010AD8B4939326
:10467000D8A4938317EC11F0180EF76E220EF66E85
:1046800086EC01F017EC11F09351E8B20FD017EC63
:1046900011F04F0E8EEC01F04E0E8EEC01F00D0E6F
:1046A0008EEC01F00A0E8EEC01F010D017EC11F038
:1046B0004F0E8EEC01F0460E8EEC01F08EEC01F008
:1046C0000D0E8EEC01F00A0E8EEC01F017EC11F0DD
:1046D000800E016E07EC00F017EC11F0AA6A0F0EC5
:1046E000A96E9351A3EC01F0C0EF28F02A0EA95D4A
:1046F00048E117EC11F017EC11F001EE88F010EE24
:10470000E6F0020EF36E030EA9EC02F0EF6A17EC6E
:1047100011F017EC11F003EE85F011EE88F0060EA3
:10472000A2EC02F0DBEC52F083C3ABF082C3AAF040
:1047300017EC11F0AB51E8AE02D0000E01D0010E23
:10474000336EAB51E8BE07D0AB5303E1AA515A0810
:1047500002E2000E01D0010E331600010FE017EC4B
:1047600011F017EC11F0AAC049F317EC11F0AA6A86
:10477000100EA96E03014951A3EC01F00001C0EF36
:1047800028F0460EA95DD8A4D9D017EC11F0E75156
:10479000076E3F0E075C3CE117EC11F017EC11F0CF
:1047A0006C50705C226E6D507158236E23C01EF0E9
:1047B00022C01DF045C317F0186A14EC02F0896F8F
:1047C00010C08AF017EC11F09351E8A608D017EC4E
:1047D00011F017EC11F0B40E895F000E8A5B17EC34
:1047E00011F0180EF76E300EF66E86EC01F0040E26
:1047F000016E030E056E8AC018F089C017F060ECD8
:1048000000F00D0E8EEC01F00A0E8EEC01F094D04B
:1048100017EC11F0E751076E300E075C000ED8B0B0
:10482000010E336EE751076E3A0E075C02E3000E8D
:1048300001D0010E3316D8B457D017EC11F017EC95
:1048400011F001EE88F010EEE6F0020EF36E030EAA
:10485000A9EC02F0EF6A17EC11F017EC11F003EE7F
:1048600085F011EE88F0060EA2EC02F0DBEC52F0BF
:1048700083C3ABF082C3AAF017EC11F0AB51E8BED2
:1048800031D0AA51AB112EE017EC11F017EC11F05A
:10489000ABC071F0AAC070F017EC11F09351E8A60C
:1048A00008D017EC11F017EC11F0B40E7026000EC2
:1048B000712217EC11F017EC11F070500301450351
:1048C000F3CF22F0F4CF23F071504503F3502326A9
:1048D00045AF02D07050235E6C502224706E6D5034
:1048E0002320716E00010FD017EC11F0E751076E15
:1048F000210E075C08E117EC11F017EC11F044C031
:1049000071F043C070F017EC11F0AA6A0C0EA96E9A
:104910007050A3EC01F07150A3EC01F017EC11F012
:10492000180EF76E460EF66E86EC01F00D0E8EEC4C
:1049300001F00A0E8EEC01F0C0EF28F0230EA95D05
:104940003AE117EC11F017EC11F0000E93B5010EDF
:10495000010AD8B49395D8A4938517EC11F0180EDA
:10496000F76E520EF66E86EC01F017EC11F09351D3
:10497000E8B40CD017EC11F0410E8EEC01F00D0EE6
:104980008EEC01F00A0E8EEC01F00BD017EC11F05A
:10499000420E8EEC01F00D0E8EEC01F00A0E8EEC44
:1049A00001F017EC11F0AA6A0F0EA96E9351A3EC57
:1049B00001F0C0EF28F0490EA95DD8A496D217ECFB
:1049C00011F00D0E8EEC01F00A0E8EEC01F0180EB7
:1049D000F76E5E0EF66E86EC01F00D0E8EEC01F0B9
:1049E0000A0E8EEC01F017EC11F0180EF76E800E27
:1049F000F66E86EC01F0040E016E056A6DC01EF0C5
:104A00006CC01DF045C317F0186A14EC02F0176E65
:104A100010C018F060EC00F0200E8EEC01F0640E77
:104A20008EEC01F0650E8EEC01F0670E8EEC01F05D
:104A30000D0E8EEC01F00A0E8EEC01F017EC11F069
:104A4000180EF76E940EF66E86EC01F0040E016EF1
:104A5000056A6FC01EF06EC01DF045C317F0186ADE
:104A600014EC02F0176E10C018F060EC00F0200E8D
:104A70008EEC01F0640E8EEC01F0650E8EEC01F010
:104A8000670E8EEC01F00D0E8EEC01F00A0E8EEC2E
:104A900001F017EC11F017EC11F06C50705C226E05
:104AA0006D507158236E23C01EF022C01DF045C307
:104AB00017F0186A14EC02F0896F10C08AF017EC36
:104AC00011F09351E8A608D017EC11F017EC11F093
:104AD000B40E895F000E8A5B17EC11F0180EF76EAA
:104AE000AA0EF66E86EC01F0040E016E056A8AC00D
:104AF00018F089C017F060EC00F0200E8EEC01F089
:104B0000640E8EEC01F0650E8EEC01F0670E8EECFB
:104B100001F00D0E8EEC01F00A0E8EEC01F017EC98
:104B200011F0180EF76EC80EF66E86EC01F0040E4A
:104B3000016E63505DEC00F0200E8EEC01F0640E0F
:104B40008EEC01F0650E8EEC01F0670E8EEC01F03C
:104B50000D0E8EEC01F00A0E8EEC01F017EC11F048
:104B6000180EF76EE80EF66E86EC01F0040E016E7C
:104B7000030149515DEC00F0200E8EEC01F0640E53
:104B80008EEC01F0650E8EEC01F0670E8EEC01F0FC
:104B90000D0E8EEC01F00A0E8EEC01F017EC11F008
:104BA000190EF76E0A0EF66E86EC01F017EC11F096
:104BB00000019351E8A20BD017EC11F04F0E8EECD0
:104BC00001F0460E8EEC01F08EEC01F008D017ECEF
:104BD00011F04F0E8EEC01F04E0E8EEC01F017EC42
:104BE00011F00D0E8EEC01F00A0E8EEC01F0190E94
:104BF000F76E1E0EF66E86EC01F0040E016E030ECB
:104C0000056E65C01EF064C01DF045C317F0186A3C
:104C100014EC02F0176E10C018F060EC00F0200EDB
:104C20008EEC01F0450E8EEC01F04C0E8EEC01F096
:104C30003A0E8EEC01F0200E8EEC01F0030E056EA4
:104C400067C01EF066C01DF045C317F0186A14EC6B
:104C500002F0176E10C018F060EC00F00D0E8EEC34
:104C600001F00A0E8EEC01F017EC11F0180EF76E41
:104C7000520EF66E86EC01F017EC11F09351E8B489
:104C800006D017EC11F0410E8EEC01F005D017ECB8
:104C900011F0420E8EEC01F017EC11F00D0E8EECBF
:104CA00001F00A0E8EEC01F0190EF76E2E0EF66E64
:104CB00086EC01F017EC11F09351E8B60FD017EC29
:104CC00011F04E0E8EEC01F06F0E8EEC01F0720EB4
:104CD0008EEC01F0640E8EEC01F011D017EC11F0A7
:104CE000530E8EEC01F06F0E8EEC01F0750E8EEC13
:104CF00001F0740E8EEC01F0680E8EEC01F017ECF2
:104D000011F00D0E8EEC01F00A0E8EEC01F0190E72
:104D1000F76E3E0EF66E86EC01F017EC11F0933153
:104D200009E317EC11F04F0E8EEC01F04E0E8EECF5
:104D300001F00AD017EC11F04F0E8EEC01F0460E88
:104D40008EEC01F08EEC01F017EC11F00D0E8EECF4
:104D500001F00A0E8EEC01F0170EF76EFE0EF66EE5
:104D600086EC01F017EC11F09351E8AA17D017EC7C
:104D700011F09351E8A809D017EC11F0180EF76E56
:104D8000080EF66E86EC01F008D017EC11F0190E43
:104D9000F76E4E0EF66E86EC01F00AD017EC11F0AD
:104DA0004F0E8EEC01F0460E8EEC01F08EEC01F011
:104DB00017EC11F00D0E8EEC01F00A0E8EEC01F0E6
:104DC000190EF76E5E0EF66E86EC01F017EC11F020
:104DD00017EC11F0030145518AEC08F02DC031F0B9
:104DE0002CC030F02BC02FF02AC02EF02D6A2C6A78
:104DF0002B6A800E2A6E7DEC07F02DC0A7F02CC028
:104E0000A6F02BC0A5F02AC0A4F017EC11F0040EF8
:104E1000016EA7C025F0A6C024F0A5C023F0A4C051
:104E200022F0010E98EC00F017EC11F0200E8EEC41
:104E300001F0640E8EEC01F0650E8EEC01F0670E51
:104E40008EEC01F017EC11F00D0E8EEC01F00A0E55
:104E50008EEC01F0190EF76E6A0EF66E86EC01F01C
:104E6000040E016E2DC325F02CC324F02BC323F0B8
:104E70002AC322F0020E98EC00F017EC11F0190E84
:104E8000F76E760EF66E86EC01F0040E016E31C3FD
:104E900025F030C324F02FC323F02EC322F0020EDE
:104EA00098EC00F017EC11F00D0E8EEC01F00A0EEC
:104EB0008EEC01F0190EF76E840EF66E86EC01F0A2
:104EC000040E016E77C325F076C324F075C323F07A
:104ED00074C322F0010E98EC00F00D0E8EEC01F080
:104EE0000A0E8EEC01F000014BD13C0EA95D54E19D
:104EF00017EC11F0190EF76E980EF66E86EC01F0B5
:104F00000D0E8EEC01F00A0E8EEC01F017EC11F094
:104F100081EC01F0A16F17EC11F017EC11F0A19BDF
:104F200017EC11F0933105E317EC11F0A1518EEC61
:104F300001F017EC11F0590EA15D2DE117EC11F005
:104F400017EC11F06DC073F06CC072F017EC11F03B
:104F500098EC3BF017EC11F03BBA0FD017EC11F0C6
:104F6000190EF76EA60EF66E86EC01F00D0E8EECA5
:104F700001F00A0E8EEC01F00ED017EC11F0190EB4
:104F8000F76EBC0EF66E86EC01F00D0E8EEC01F0A5
:104F90000A0E8EEC01F0F4D05E0EA95D54E117EC20
:104FA00011F0190EF76E980EF66E86EC01F00D0EEC
:104FB0008EEC01F00A0E8EEC01F017EC11F081EC92
:104FC00001F0A16F17EC11F017EC11F0A19B17EC99
:104FD00011F0933105E317EC11F0A1518EEC01F0C3
:104FE00017EC11F0590EA15D2DE117EC11F017EC43
:104FF00011F06FC075F06EC074F017EC11F0B2ECE8
:105000003CF017EC11F03BBC0FD017EC11F0190E6F
:10501000F76ED60EF66E86EC01F00D0E8EEC01F0FA
:105020000A0E8EEC01F00ED017EC11F0190EF76E8F
:10503000EE0EF66E86EC01F00D0E8EEC01F00A0E0F
:105040008EEC01F09DD02F0EA95D3FE117EC11F021
:10505000E951076E2E0E075C0FE017EC11F01A0EE7
:10506000F76E0A0EF66E86EC01F00D0E8EEC01F076
:105070000A0E8EEC01F028D017EC11F017EC11F0AD
:1050800001EE88F010EEE6F0020EF36E050EA9ECCC
:1050900002F0EF6A17EC11F017EC11F001EE88F056
:1050A00016EC00F01AC02DF019C02CF018C02BF02F
:1050B00017C02AF08EEC08F02DC02DF32CC02CF375
:1050C0002BC02BF32AC02AF35BD0220EA95D3FE14F
:1050D00017EC11F0EA51076E2E0E075C0FE017EC8B
:1050E00011F01A0EF76E1A0EF66E86EC01F00D0E28
:1050F0008EEC01F00A0E8EEC01F028D017EC11F0C6
:1051000017EC11F001EE88F010EEE6F0020EF36EEF
:10511000060EA9EC02F0EF6A17EC11F017EC11F093
:1051200001EE88F016EC00F01AC02DF019C02CF03A
:1051300018C02BF017C02AF08EEC08F02DC031F308
:105140002CC030F32BC02FF32AC02EF319D017EC4C
:1051500011F0933115E317EC11F03F0E8EEC01F0D6
:105160003E0E8EEC01F000EEE6F0EE5003E08EEC29
:1051700001F0FBD70D0E8EEC01F00A0E8EEC01F063
:1051800017EC11F017EC11F000EEE6F0EF6A17ECF7
:1051900011F03BB843D117EC11F0000E3AB0010EFC
:1051A000336E010E3BBA000E3316D8B476D017EC2E
:1051B00011F043505B5C44505C5844505C18D8B0CC
:1051C000800A1EE617EC11F081A608D017EC11F04A
:1051D00093968A9617EC11F0D0EC3DF017EC11F095
:1051E00017EC11F03D9C17EC11F017EC11F03D8E0F
:1051F00017EC11F093988A8817EC11F095968C862D
:1052000017EC11F05B50435C5C50445844505C1800
:10521000D8B0800A1EE617EC11F081A808D017EC70
:1052200011F093988A9817EC11F0D0EC3DF017EC40
:1052300011F017EC11F03D9E17EC11F017EC11F086
:105240003D8C17EC11F093968A8617EC11F0959629
:105250008C8617EC11F05C50445C03E15B50435CBE
:1052600002E0000E01D0010E336E000E3BB8010EBD
:105270003312000112E017EC11F093968A9617ECA6
:1052800011F093988A9817EC11F017EC11F03A90FE
:1052900017EC11F017EC11F03A9817EC11F0010E21
:1052A00093B3000E336E42AE02D0000E01D0010E59
:1052B00033164150BE5D4250BF594250BF19D8B05D
:1052C000800A02E6000E01D0010E3316D8B48DD04C
:1052D00017EC11F0010E3BBC000E336E000E3AB21B
:1052E000010E3316D8B480D017EC11F017EC11F082
:1052F0006E50455C496E6F5046584A6E17EC11F07F
:105300004950415C4A5042584A504218D8B0800A2D
:105310001EE617EC11F081AA08D017EC11F0939A51
:105320008A9A17EC11F0D0EC3DF017EC11F017EC65
:1053300011F03E9017EC11F017EC11F03E8217ECD3
:1053400011F0939C8A8C17EC11F095968C8617ECD3
:1053500011F04150495C42504A584A504218D8B066
:10536000800A1EE617EC11F081AC08D017EC11F0A2
:10537000939C8A9C17EC11F0D0EC3DF017EC11F0E7
:1053800017EC11F03E9217EC11F017EC11F03E8083
:1053900017EC11F0939A8A8A17EC11F095968C8687
:1053A00017EC11F042504A5C03E14150495C02E0C5
:1053B000000E01D0010E336E000E3BB8010E331209
:1053C000000112E017EC11F0939C8A9C17EC11F08D
:1053D000939A8A9A17EC11F017EC11F03A9217ECA5
:1053E00011F017EC11F03A9A05D017EC11F017EC08
:1053F00011F03A9217EC11F0010E3AB0000E336E34
:10540000010E3AB2000E331609E017EC11F0959632
:105410008C9617EC11F017EC11F03E9817EC11F088
:105420002FEF11F017EC11F09351E8B283EF2DF04C
:1054300017EC11F03BBCC9D117EC11F03CBA60D1AC
:1054400017EC11F017EC11F0FE0E49144B6EFF0E25
:105450004A144C6E17EC11F04CAEA8D017EC11F0BA
:10546000800E016E0FEC00F0450E34EC01F04C0E96
:1054700034EC01F03A0E34EC01F0200E34EC01F083
:105480002D0E34EC01F017EC11F04CC008F04BC0BD
:1054900007F008AE03D0076CE86A0856C051075CF5
:1054A000C15108580850C119D8B0800A06E617EC57
:1054B00011F0200E34EC01F021D017EC11F017ECB4
:1054C00011F04CC008F04BC007F008AE03D0076CD9
:1054D000E86A085608C01EF007C01DF0C1C018F0E9
:1054E000C0C017F014EC02F0956F17EC11F0800EAD
:1054F000016E010E056E95515EEC00F017EC11F097
:10550000800E016E010E056E4CC008F04BC007F016
:1055100008AE03D0076CE86A085608C01EF007C042
:105520001DF045C317F0186A14EC02F0176E10C096
:1055300018F060EC00F017EC11F02E0E34EC01F0D6
:1055400017EC11F017EC11F04CC008F04BC007F04D
:1055500008AE03D0076CE86A085608C01EF007C002
:105560001DF045C317F0186A14EC02F013C095F053
:1055700017EC11F017EC11F095510A0DF3CF22F052
:10558000F4CF23F023C010F022C00FF0146A45C3FB
:1055900013F0FDEC01F0956F17EC11F0800E016E29
:1055A000010E056E95515EEC00F0A9D017EC11F0DC
:1055B000800E016E0FEC00F0450E34EC01F04C0E45
:1055C00034EC01F03A0E34EC01F0200E34EC01F032
:1055D00017EC11F0C2514B5CC3514C584C50C319DD
:1055E000D8B0800A06E617EC11F0200E34EC01F07A
:1055F00018D017EC11F017EC11F04CC01EF04BC096
:105600001DF0C3C018F0C2C017F014EC02F0956F83
:1056100017EC11F0800E016E010E056E95515EECD7
:1056200000F017EC11F0C0514B5CC1514C584C507C
:10563000C119D8B0800A06E617EC11F0200E34EC40
:1056400001F018D017EC11F017EC11F04CC01EF05F
:105650004BC01DF0C1C018F0C0C017F014EC02F030
:10566000956F17EC11F0800E016E010E056E9551CD
:105670005EEC00F017EC11F0800E016E010E056E6D
:105680004CC01EF04BC01DF045C317F0186A14EC57
:1056900002F0176E10C018F060EC00F017EC11F07B
:1056A0002E0E34EC01F017EC11F017EC11F04CC099
:1056B0001EF04BC01DF045C317F0186A14EC02F041
:1056C00013C095F017EC11F017EC11F095510A0D7D
:1056D000F3CF22F0F4CF23F023C010F022C00FF05C
:1056E000146A45C313F0FDEC01F0956F17EC11F04F
:1056F000800E016E010E056E95515EEC00F064D0D7
:1057000017EC11F017EC11F02D6A2C6A200E2B6E9D
:10571000820E2A6E27C331F026C330F025C32FF046
:1057200024C32EF0E3EC07F031EC08F04B6E2BC0F5
:105730004CF017EC11F0800E016E0FEC00F0450EEE
:1057400034EC01F04C0E34EC01F03A0E34EC01F084
:10575000200E34EC01F034EC01F017EC11F027C30B
:105760002DF026C32CF025C32BF024C32AF0316A78
:10577000306A200E2F6E820E2E6E33EC06F001087A
:1057800005E017EC11F0200E34EC01F017EC11F0ED
:10579000800E016E056A4CC01EF04BC01DF0186AE9
:1057A0000A0E176E14EC02F0176E10C018F060ECC1
:1057B00000F02E0E34EC01F0010E056E4CC018F016
:1057C0004BC017F060EC00F00CD017EC11F0800E1D
:1057D000016E0FEC00F01A0EF76E2A0EF66E2CEC2E
:1057E00001F017EC11F08AAC05D017EC11F0000EA7
:1057F00034EC01F017EC11F08AAA05D017EC11F087
:10580000010E34EC01F017EC11F0010E8ABA000E13
:10581000336E010E8ABC000E331605E017EC11F052
:10582000200E34EC01F017EC11F08AA805D017EC2B
:1058300011F0030E34EC01F017EC11F08AA605D03C
:1058400017EC11F0020E34EC01F017EC11F0010E20
:105850008AB6000E336E010E8AB8000E331605E0CC
:1058600017EC11F0200E34EC01F017EC11F03CBAFB
:10587000CAD017EC11F03BBABDD017EC11F03CBA0E
:105880000BD017EC11F017EC11F0FE0E47144D6E13
:10589000FF0E48144E6E08D017EC11F017EC11F003
:1058A00040C04EF03FC04DF017EC11F0410E34EC0B
:1058B00001F05A0E34EC01F03A0E34EC01F0200EF7
:1058C00034EC01F017EC11F0C2514D5CC3514E584D
:1058D0004E50C319D8B0800A06E617EC11F0200E1E
:1058E00034EC01F018D017EC11F017EC11F04EC0A9
:1058F0001EF04DC01DF0C3C018F0C2C017F014EC6C
:1059000002F0956F17EC11F0800E016E010E056E1E
:1059100095515EEC00F017EC11F0C0514D5CC15197
:105920004E584E50C119D8B0800A06E617EC11F057
:10593000200E34EC01F018D017EC11F017EC11F038
:105940004EC01EF04DC01DF0C1C018F0C0C017F011
:1059500014EC02F0956F17EC11F0800E016E010E41
:10596000056E95515EEC00F017EC11F0800E016EA3
:10597000010E056E4EC01EF04DC01DF045C317F060
:10598000186A14EC02F0176E10C018F060EC00F00A
:1059900017EC11F02E0E34EC01F017EC11F017ECAF
:1059A00011F04EC01EF04DC01DF045C317F0186A2F
:1059B00014EC02F013C095F017EC11F017EC11F095
:1059C00095510A0DF3CF22F0F4CF23F023C010F04D
:1059D00022C00FF0146A45C313F0FDEC01F0956F7F
:1059E00017EC11F0800E016E010E056E95515EEC04
:1059F00000F008D017EC11F01A0EF76E340EF66EA8
:105A00002CEC01F077D017EC11F017EC11F02D6AA7
:105A10002C6A200E2B6E820E2A6E23C331F022C315
:105A200030F021C32FF020C32EF0E3EC07F031EC6F
:105A300008F04D6E2BC04EF017EC11F0410E34EC17
:105A400001F05A0E34EC01F03A0E34EC01F0200E65
:105A500034EC01F017EC11F023C32DF022C32CF02D
:105A600021C32BF020C32AF0316A306A480E2F6E12
:105A7000850E2E6E33EC06F0010805E017EC11F0F0
:105A8000200E34EC01F017EC11F023C32DF022C3EB
:105A90002CF021C32BF020C32AF0316A306A200E8B
:105AA0002F6E820E2E6E33EC06F0010805E017EC27
:105AB00011F0200E34EC01F017EC11F0800E016EA5
:105AC000056A4EC01EF04DC01DF0186A0A0E176E12
:105AD00014EC02F0176E10C018F060EC00F02E0EFF
:105AE00034EC01F0010E056E4EC018F04DC017F0F9
:105AF00060EC00F017EC11F01A0EF76E3E0EF66E29
:105B00002CEC01F006D117EC11F03BBAEED017ECFB
:105B100011F03CBA0BD017EC11F017EC11F0FE0E9F
:105B200047144D6EFF0E48144E6E08D017EC11F05E
:105B300017EC11F040C04EF03FC04DF017EC11F0E3
:105B4000800E016E0FEC00F01A0EF76E540EF66E1A
:105B50002CEC01F017EC11F0C2514D5CC3514E58C2
:105B60004E50C319D8B0800A06E617EC11F0200E8B
:105B700034EC01F018D017EC11F017EC11F04EC016
:105B80001EF04DC01DF0C3C018F0C2C017F014ECD9
:105B900002F0956F17EC11F0800E016E010E056E8C
:105BA00095515EEC00F017EC11F0C0514D5CC15105
:105BB0004E584E50C119D8B0800A06E617EC11F0C5
:105BC000200E34EC01F018D017EC11F017EC11F0A6
:105BD0004EC01EF04DC01DF0C1C018F0C0C017F07F
:105BE00014EC02F0956F17EC11F0800E016E010EAF
:105BF000056E95515EEC00F017EC11F0800E016E11
:105C0000010E056E4EC01EF04DC01DF045C317F0CD
:105C1000186A14EC02F0176E10C018F060EC00F077
:105C200017EC11F02E0E34EC01F017EC11F017EC1C
:105C300011F04EC01EF04DC01DF045C317F0186A9C
:105C400014EC02F013C095F017EC11F017EC11F002
:105C500095510A0DF3CF22F0F4CF23F023C010F0BA
:105C600022C00FF0146A45C313F0FDEC01F0956FEC
:105C700017EC11F0800E016E010E056E95515EEC71
:105C800000F017EC11F0200E34EC01F0640E34EC4F
:105C900001F0650E34EC01F0670E34EC01F0200EDB
:105CA00034EC01F017EC11F08AA805D017EC11F0D4
:105CB000030E34EC01F017EC11F08AA605D017ECB6
:105CC00011F0020E34EC01F017EC11F0010E8AB65F
:105CD000000E336E010E8AB8000E331605E017EC85
:105CE00011F0200E34EC01F00CD017EC11F0800E06
:105CF000016E0FEC00F01A0EF76E5E0EF66E2CECD5
:105D000001F017EC11F01A0EF76E740EF66E2CEC13
:105D100001F017EF11F017EC11F093968A9617EC3B
:105D200011F093988A9817EC11F0939C8A9C17ECC9
:105D300011F0939A8A9A17EC11F095968C9617ECBD
:105D400011F017EC11F03E9817EC11F017EC11F070
:105D500042C0B5F041C0B4F017EC11F017EC11F0EF
:105D600040C0B3F03FC0B2F017EC11F0AF6B010EC2
:105D7000AE6FAF5312E10B0EAE5D0FE217EC11F0F8
:105D8000050EBAEC01F017EC11F017EC48F017EC27
:105D900011F0AE2B000EAF23ECE317EC11F082B242
:105DA0008DD017EC11F0010E3AB4000E336E010ED7
:105DB0003AB6000E33160CE017EC11F017EC11F0A8
:105DC000000E3BB8010E010AD8B43B98D8A43B881A
:105DD00017EC11F017EC11F03A9017EC11F017ECEA
:105DE00011F03A9217EC11F017EC11F03A9417EC0D
:105DF00011F017EC11F03A9617EC11F017EC11F0C6
:105E000044C050F043C04FF017EC11F017EC11F004
:105E100046C052F045C051F017EC11F017EC11F0EC
:105E20003B9A17EC11F017EC11F03B9C17EC11F0BA
:105E300017EC11F00301416B17EC11F017EC11F0A6
:105E40000301426B17EC11F017EC11F000EEE6F0D5
:105E5000EF6A17EC11F017EC11F03D9817EC11F008
:105E600017EC11F03BB882803BA8829017EC11F040
:105E700017EC11F00001B16BB06B17EC11F082B2AE
:105E80001DD017EC11F017EC11F0B04BB12B17EC43
:105E900011F0030E106E200EC8EC01F017EC11F09B
:105EA000050EB15D0AE303E1DD0EB05D06E317EC1C
:105EB00011F0000105D817EF11F0E1D717EF11F03D
:105EC00017EC11F017EC11F0829017EC11F017ECB1
:105ED00011F03B9817EC11F017EC11F0906B17ECE8
:105EE00011F017EC11F0839217EC11F017EC11F090
:105EF000839017EC11F0800E016E0FEC00F01A0E7B
:105F0000F76E8A0EF66E2CEC01F017EC11F01A0EFB
:105F1000F76EA00EF66E2CEC01F017EC11F082A2D9
:105F2000FED717EC11F017EC11F00301140E446FBB
:105F300017EC11F017EC11F048C01EF047C01DF02F
:105F400045C317F0186A14EC02F0576E10C058F0F1
:105F500017EC11F017EC11F0585003014503F3CF83
:105F600058F057504503F3CF57F0F450582645AF3B
:105F700002D05750585E17EC11F017EC11F04AC0E0
:105F80005AF049C059F017EC11F017EC11F065C048
:105F900069F064C068F017EC11F017EC11F067C0FD
:105FA0006BF066C06AF017EC11F017EC11F06DC0E1
:105FB00073F06CC072F017EC11F017EC11F06FC0B9
:105FC00075F06EC074F017EC11F017EC11F06C5016
:105FD000705C766E6D507158776E17EC11F00001A1
:105FE0009351E8A60AD017EC11F017EC11F0BA5152
:105FF000765C766EBB517758776E17EC11F017EC24
:1060000011F03B8E93A13B9E17EC11F017EC11F0B1
:106010003C8093A33C9017EC11F017EC11F03C86F8
:1060200093A53C9617EC11F017EC11F063C0A8F0A3
:1060300017EC11F017EC11F03C8293A73C9217EC8F
:1060400011F017EC11F03C8493A93C9417EC11F07B
:1060500017EC11F03C8893AB3C9817EC11F017EC5F
:1060600011F03C8C3CAA3C9C17EC11F017EC11F0A1
:1060700045C37AF017EC11F017EC11F049C378F032
:10608000796A17EC11F017EC11F03B8493AD3B9457
:1060900017EC11F017EC11F03B8693AF3B9617EC21
:1060A00011F017EC11F02DC37EF02CC37DF02BC343
:1060B0007CF02AC37BF017EC11F017EC11F031C320
:1060C00082F030C381F02FC380F02EC37FF017EC35
:1060D00011F017EC11F033C384F032C383F017ECE6
:1060E00011F017EC11F0A85103014503F4CFBFF0F4
:1060F000F3CFBEF017EC11F0000117EC11F082B4F1
:1061000021D017EC11F0140EBAEC01F017EC11F0DD
:1061100082B417D017EC11F017EC11F08F0717ECC1
:1061200011F0010E8F5D06E217EC11F017EC11F083
:10613000160E8F6F17EC11F017EC11F00301140E0F
:10614000446F000117EC11F082B621D017EC11F06A
:10615000140EBAEC01F017EC11F082B617D017EC60
:1061600011F017EC11F08F2B17EC11F0170E8F5D5B
:1061700006E317EC11F017EC11F0010E8F6F17EC1E
:1061800011F017EC11F00301140E446F000117EC2D
:1061900011F080BC16D017EC11F0140EBAEC01F01F
:1061A00017EC11F080BC06D017EC11F017EC11F0D1
:1061B000FF0E906F17EC11F017EC11F00301140EA5
:1061C000446F000117EC11F080BE16D017EC11F0EF
:1061D000140EBAEC01F017EC11F080BE06D017ECEB
:1061E00011F017EC11F0010E906F17EC11F017EC95
:1061F00011F00301140E446F000117EC11F0010EB1
:1062000082B2000E336E010E03014453D8A4000E77
:1062100033120001D8B425D217EC11F00E0E8F5DA9
:10622000010ED8A4000E336E010E82B2000E33169A
:106230000EE017EC11F017EC11F03C9817EC11F090
:1062400017EC11F00301140E446F00010AD217EC91
:1062500011F017EC11F058C040F057C03FF017ECA8
:1062600011F017EC11F05AC042F059C041F017EC90
:1062700011F0000E63BEFF0E425C07E0425063184F
:10628000D8B0800A800B2CE003D04150635C28E238
:1062900017EC11F017EC11F041500001BA5D416E9E
:1062A0004250BB59426E17EC11F017EC11F0BA5185
:1062B0003F26BB51402217EC11F0BC513F5CBD5151
:1062C00040584050BD19D8B0800A0AE717EC11F0C9
:1062D00017EC11F0BC513F5C3F6EBD514058406E11
:1062E00017EC11F017EC11F069C065F068C064F0AC
:1062F00017EC11F017EC11F06BC067F06AC066F094
:1063000017EC11F017EC11F073C06DF072C06CF067
:1063100017EC11F017EC11F075C06FF074C06EF04F
:1063200017EC11F017EC11F072507624706E735068
:106330007720716E17EC11F09351E8A608D017EC96
:1063400011F017EC11F0BA517026BB51712217EC05
:1063500011F017EC11F093813BAE939117EC11F013
:1063600017EC11F093833CA0939317EC11F017EC0A
:1063700011F093853CA6939517EC11F017EC11F0F2
:10638000A8C063F017EC11F017EC11F093873CA252
:10639000939717EC11F017EC11F093893CA49399A3
:1063A00017EC11F017EC11F0938B3CA8939B17ECB2
:1063B00011F017EC11F03C8A3CAC3C9A17EC11F050
:1063C00017EC11F084C033F383C032F317EC11F0F3
:1063D00017EC11F07AC045F317EC11F017EC11F03F
:1063E00003014551B40DF3CFBAF0F4CFBBF017EC75
:1063F00011F017EC11F003014551680DF3CFBCF01B
:10640000F4CFBDF00001BD2717EC11F017EC11F02F
:10641000635003014503F4CFBFF0F3CFBEF017EC98
:1064200011F017EC11F0030145510A0DF3CFC0F044
:10643000F4CFC1F017EC11F017EC11F00301455146
:10644000640DF3CFC2F0F4CFC3F017EC11F017ECEA
:1064500011F078C049F317EC11F017EC11F00001BE
:10646000938D3BA4939D17EC11F017EC11F0938FD3
:106470003BA6939F17EC11F017EC11F0635003014A
:106480004503F4CFBFF0F3CFBEF017EC11F0AA6ACA
:10649000040EA96E6450A3EC01F06550A3EC01F06A
:1064A00017EC11F0AA6A060EA96E6650A3EC01F073
:1064B0006750A3EC01F017EC11F0AA6A080EA96E60
:1064C0006C50A3EC01F06D50A3EC01F017EC11F04F
:1064D000AA6A0A0EA96E6E50A3EC01F06F50A3ECED
:1064E00001F017EC11F0AA6A0C0EA96E7050A3EC23
:1064F00001F07150A3EC01F017EC11F0AA6A0E0E36
:10650000A96E6350A3EC01F017EC11F0AA6A0F0E0C
:10651000A96E00019351A3EC01F017EC11F0AA6AE7
:10652000100EA96E03014951A3EC01F017EC11F014
:10653000AA6A110EA96E03014551A3EC01F017ECF4
:1065400011F0AA6A120EA96E03012A51A3EC01F000
:1065500003012B51A3EC01F003012C51A3EC01F03A
:1065600003012D51A3EC01F017EC11F0AA6A160EED
:10657000A96E03012E51A3EC01F003012F51A3ECEE
:1065800001F003013051A3EC01F003013151A3EC00
:1065900001F017EC11F0AA6A1A0EA96E030132512C
:1065A000A3EC01F003013351A3EC01F017EC11F05F
:1065B000800E016E07EC00F017EC11F0000112ECF8
:1065C0002AF017EC11F082A2FED717EC11F0000EA2
:1065D0003AB0010E336E000E3AB2010E331209E0EA
:1065E00017EC11F095968C8617EC11F017EC11F062
:1065F0003E8817EC11F09351E8A620D017EC11F06B
:1066000017EC11F0BA513F245B6EBB5140205C6E19
:1066100017EC11F05B50BC5D5C50BD595C50BD196E
:10662000D8B0800A0AE617EC11F017EC11F0BC5153
:106630005B5C5B6EBD515C585C6E08D017EC11F072
:1066400017EC11F040C05CF03FC05BF017EC11F0AC
:10665000D2EC46F017EC11F017EC11F03B9817EF65
:1066600011F017EC11F0010E8F5DD8A46ED017EC6D
:1066700011F017EC11F0905103014503F3CF22F014
:10668000F4CF23F045AF01D0235E000190AF03D0DB
:1066900003014551235E225057262350582217EC00
:1066A00011F00001905305E017EC11F017EC11F018
:1066B0003A8017EC11F05750BC5D5850BD595850F6
:1066C000BD19D8B0800A0AE617EC11F017EC11F0EA
:1066D000BC51575C576EBD515858586E17EC11F0AD
:1066E00058AE08D017EC11F017EC11F0BC5157263A
:1066F000BD51582217EC11F0800E016E0FEC00F026
:106700001A0EF76EB60EF66E2CEC01F017EC11F0C7
:10671000800E016E030E056E58C01EF057C01DF0AE
:1067200045C317F0186A14EC02F0176E10C018F089
:1067300060EC00F017EC11F0050E34EC01F017ECF2
:1067400011F0E4EC51F020EF3BF0020E8F5DD8A485
:106750006ED017EC11F017EC11F0905103014503C6
:10676000F3CF22F0F4CF23F045AF01D0235E000138
:1067700090AF03D003014551235E22505926235088
:106780005A2217EC11F00001905305E017EC11F0BC
:1067900017EC11F03A8217EC11F05950BE5D5A50C7
:1067A000BF595A50BF19D8B0800A0BE617EC11F048
:1067B00017EC11F0A85103014503F4CF5AF0F3CFC1
:1067C00059F0000117EC11F05AAE06D017EC11F099
:1067D00017EC11F05A6A596A17EC11F0800E016E2D
:1067E0000FEC00F01A0EF76EC80EF66E2CEC01F0EE
:1067F00017EC11F0800E016E030E056E5AC01EF0EC
:1068000059C01DF045C317F0186A14EC02F0176E5A
:1068100010C018F060EC00F017EC11F0050E34EC2D
:1068200001F017EC11F0E4EC51F020EF3BF0030E17
:106830008F5DD8A461D017EC11F017EC11F09051D6
:1068400003014503F3CF22F0F4CF23F045AF01D08D
:10685000235E000190AF03D003014551235E225017
:1068600068262350692217EC11F068500001BC5DC6
:106870006950BD596950BD19D8B0800A08E617ECB7
:1068800011F017EC11F0BDC069F0BCC068F017EC56
:1068900011F069AE06D017EC11F017EC11F0696A2F
:1068A000686A17EC11F0800E016E0FEC00F01A0E02
:1068B000F76EDA0EF66E2CEC01F017EC11F0800E8C
:1068C000016E030E056E69C01EF068C01DF045C361
:1068D00017F0186A14EC02F0176E10C018F060EC94
:1068E00000F017EC11F0050E34EC01F017EC11F08C
:1068F000E4EC51F020EF3BF0040E8F5DD8A465D09E
:1069000017EC11F017EC11F0905103014503F3CF90
:1069100022F0F4CF23F045AF01D0235E000190AF09
:1069200003D003014551235E22506A2623506B2277
:1069300017EC11F06A500001BE5D6B50BF596B50EF
:10694000BF19D8B0800A0BE617EC11F017EC11F064
:10695000A85103014503F4CF6BF0F3CF6AF00001B7
:1069600017EC11F06BAE06D017EC11F017EC11F02C
:106970006B6A6A6A17EC11F0800E016E0FEC00F082
:106980001A0EF76EEC0EF66E2CEC01F017EC11F00F
:10699000800E016E030E056E6BC01EF06AC01DF006
:1069A00045C317F0186A14EC02F0176E10C018F007
:1069B00060EC00F017EC11F0050E34EC01F017EC70
:1069C00011F0E4EC51F020EF3BF0050E8F5DD8A400
:1069D00061D017EC11F017EC11F090510301450351
:1069E000F3CF22F0F4CF23F045AF01D0235E0001B6
:1069F00090AF03D003014551235E225072262350ED
:106A0000732217EC11F072500001C45D7350C55928
:106A10007350C519D8B0800A08E617EC11F017ECCE
:106A200011F0C5C073F0C4C072F017EC11F073AE72
:106A300006D017EC11F017EC11F0736A726A17ECBC
:106A400011F0800E016E0FEC00F01A0EF76EFE0EC4
:106A5000F66E2CEC01F017EC11F0800E016E030EB7
:106A6000056E73C01EF072C01DF045C317F0186AA2
:106A700014EC02F0176E10C018F05BEC00F017EC8D
:106A800011F0050E34EC01F017EC11F0E4EC51F0CC
:106A900020EF3BF0060E8F5DD8A461D017EC11F00B
:106AA00017EC11F0905103014503F3CF22F0F4CF1E
:106AB00023F045AF01D0235E000190AF03D0030166
:106AC0004551235E225074262350752217EC11F095
:106AD00074500001C65D7550C7597550C719D8B0BC
:106AE000800A08E617EC11F017EC11F0C7C075F03A
:106AF000C6C074F017EC11F075AE06D017EC11F0AB
:106B000017EC11F0756A746A17EC11F0800E016EC3
:106B10000FEC00F01B0EF76E100EF66E2CEC01F071
:106B200017EC11F0800E016E030E056E75C01EF09D
:106B300074C01DF045C317F0186A14EC02F0176E0C
:106B400010C018F05BEC00F017EC11F0050E34ECFF
:106B500001F017EC11F0E4EC51F020EF3BF0070EE0
:106B60008F5DD8A4D5D017EC11F017EC11F090512F
:106B700003014503F3CF22F0F4CF23F045AF01D05A
:106B8000235E000190AF03D003014551235E2250E4
:106B900076262350772217EC11F000019351E8B6C6
:106BA0004BD017EC11F0BC51765CBD517758775043
:106BB000BD19D8B0800A08E617EC11F017EC11F0F7
:106BC000BDC077F0BCC076F017EC11F00301455161
:106BD000A40DF3CF07F0F4CF08F0096A0A6A455113
:106BE000010DF3500826F4500922000E0A2276C047
:106BF0000FF077C010F0000E10BEFF0E116E126E77
:106C00000F50075C105008581150095812500A587C
:106C10000A501218D8B0800A00010CE617EC11F0E7
:106C200017EC11F003014551A40DF3CF76F0F4CF2A
:106C300077F07726000141D017EC11F0BA51765C5D
:106C4000BB5177587750BB19D8B0800A08E617ECCB
:106C500011F017EC11F0BBC077F0BAC076F017EC6A
:106C600011F003014551F00DF3CF07F0F4CF08F018
:106C7000096A0A6A76C00FF077C010F0000E10BEE5
:106C8000FF0E116E126E0F50075C10500858115015
:106C9000095812500A580A501218D8B0800A000138
:106CA0000BE617EC11F017EC11F003014551F00D54
:106CB000F3CF76F0F4CF77F0000117EC11F0800EEF
:106CC000016E0FEC00F01B0EF76E220EF66E2CEC30
:106CD00001F017EC11F0800E016E030E056E77C007
:106CE0001EF076C01DF045C317F0186A14EC02F0D0
:106CF000176E10C018F060EC00F017EC11F0050EE4
:106D000034EC01F017EC11F0E4EC51F020EF3BF023
:106D1000080E8F5D2FE117EC11F017EC11F0905178
:106D20007824786E000E90BFFF0E7920796E17ECF4
:106D300011F0800E016E0FEC00F01B0EF76E340E9A
:106D4000F66E2CEC01F017EC11F0800E016E030EC4
:106D5000056E79C018F078C017F060EC00F017EC01
:106D600011F0050E34EC01F017EC11F0E4EC51F0E9
:106D700020EF3BF0090E8F5D42E117EC11F09051CE
:106D8000E8BE07D0905305E017EC11F017EC11F0B6
:106D90003B8E17EC11F09051E8AE05D017EC11F0D6
:106DA00017EC11F03B9E17EC11F0800E016E0FEC0A
:106DB00000F01B0EF76E460EF66E2CEC01F017EC91
:106DC00011F03BAE0CD017EC11F0200E34EC01F0BA
:106DD0004F0E34EC01F04E0E34EC01F00AD017ECFB
:106DE00011F04F0E34EC01F0460E34EC01F034ECAF
:106DF00001F017EC11F01FEC52F020EF3BF00A0EFF
:106E00008F5D42E117EC11F09051E8BE07D090532E
:106E100005E017EC11F017EC11F03C9017EC11F0B5
:106E20009051E8AE05D017EC11F017EC11F03C8052
:106E300017EC11F0800E016E0FEC00F01B0EF76ED8
:106E4000580EF66E2CEC01F017EC11F03CA00BD0B4
:106E500017EC11F04F0E34EC01F0460E34EC01F05B
:106E600034EC01F00BD017EC11F0200E34EC01F0F3
:106E70004F0E34EC01F04E0E34EC01F017EC11F033
:106E80001FEC52F020EF3BF00B0E8F5D57E117EC3B
:106E900011F09051E8BE07D0905305E017EC11F0C7
:106EA00017EC11F03C8617EC11F09051E8AE05D0CC
:106EB00017EC11F017EC11F03C9617EC11F0800E66
:106EC000016E0FEC00F01B0EF76E6A0EF66E2CECE6
:106ED00001F017EC11F03CA606D017EC11F0420EB1
:106EE00034EC01F005D017EC11F0410E34EC01F058
:106EF00017EC11F0200E34EC01F0000E34EC01F030
:106F0000200E34EC01F04D0E34EC01F0200E34EC88
:106F100001F0010E34EC01F0200E34EC01F034EC01
:106F200001F034EC01F0040E34EC01F01B0EF76EAE
:106F30007E0EF66E2CEC01F020EF3BF00C0E8F5D18
:106F4000D8A464D017EC11F09051E8BE08D090534B
:106F500006E017EC11F017EC11F0B40EA86F17EC67
:106F600011F09051E8AE06D017EC11F017EC11F0CB
:106F70005A0EA86F17EC11F017EC11F0A85103018D
:106F80004503F4CFBFF0F3CFBEF017EC11F0800E45
:106F9000016E0FEC00F01B0EF76E8A0EF66E2CECF5
:106FA00001F017EC11F0800E016E030E056E00016A
:106FB000A8515EEC00F017EC11F0050E34EC01F076
:106FC00017EC11F0200E34EC01F0000E34EC01F05F
:106FD000200E34EC01F04D0E34EC01F0200E34ECB8
:106FE00001F0010E34EC01F0200E34EC01F034EC31
:106FF00001F034EC01F0040E34EC01F01B0EF76EDE
:107000009C0EF66E2CEC01F020EF3BF00D0E8F5D28
:10701000D8A45CD017EC11F09051E8BE07D0905383
:1070200005E017EC11F017EC11F03C8217EC11F0B1
:107030009051E8AE05D017EC11F017EC11F03C922E
:1070400017EC11F0800E016E0FEC00F01B0EF76EC6
:10705000A80EF66E2CEC01F017EC11F03CB209D042
:1070600017EC11F01B0EF76EB80EF66E2CEC01F05B
:1070700008D017EC11F01B0EF76EC00EF66E2CEC5C
:1070800001F017EC11F0200E34EC01F0000E34EC9E
:1070900001F0200E34EC01F04D0E34EC01F0200E26
:1070A00034EC01F0010E34EC01F0200E34EC01F070
:1070B00034EC01F034EC01F0040E34EC01F01B0E62
:1070C000F76EC80EF66E2CEC01F0BAD20E0E8F5D84
:1070D000D8A469D017EC11F09051E8BE0CD09053B1
:1070E0000AE017EC11F017EC11F03C8417EC11F0EA
:1070F00017EC11F03C8817EC11F09051E8AE0AD073
:1071000017EC11F017EC11F03C9417EC11F017ECA0
:1071100011F03C8817EC11F0800E016E0FEC00F0BE
:107120001B0EF76ED40EF66E2CEC01F017EC11F07E
:107130003CB809D017EC11F01B0EF76EDE0EF66EA0
:107140002CEC01F015D017EC11F03CB409D017EC81
:1071500011F01B0EF76EEA0EF66E2CEC01F008D063
:1071600017EC11F01B0EF76EF60EF66E2CEC01F01C
:1071700017EC11F0200E34EC01F0000E34EC01F0AD
:10718000200E34EC01F04D0E34EC01F0200E34EC06
:1071900001F0010E34EC01F01C0EF76E020EF66EDB
:1071A0002CEC01F04DD20F0E8F5D2DE117EC11F09C
:1071B000800E016E0FEC00F01C0EF76E120EF66ED4
:1071C0002CEC01F077C325F076C324F075C323F0CF
:1071D00074C322F0010E98EC00F0200E34EC01F0A4
:1071E00034EC01F034EC01F034EC01F034EC01F05B
:1071F00017EC11F0800E016E160E046E020E186E62
:107200001CEC01F01DD2100E8F5DD8A499D017ECA4
:1072100011F09051E8BE23D0905321E017EC11F00B
:10722000040E7A5C06E117EC11F017EC11F0020E77
:107230007A6E17EC11F00A0E7A5C06E117EC11F089
:1072400017EC11F0040E7A6E17EC11F0140E7A5C44
:1072500006E117EC11F017EC11F00A0E7A6E17EC3C
:1072600011F09051E8AE21D017EC11F00A0E7A5CC3
:1072700006E117EC11F017EC11F0140E7A6E17EC12
:1072800011F0040E7A5C06E117EC11F017EC11F026
:107290000A0E7A6E17EC11F0020E7A5C06E117EC1A
:1072A00011F017EC11F0040E7A6E17EC11F0800E4D
:1072B000016E0FEC00F01C0EF76E200EF66E2CEC3B
:1072C00001F017EC11F0140E7A5C09E117EC11F0E3
:1072D0001C0EF76E2C0EF66E2CEC01F024D017EC81
:1072E00011F00A0E7A5C09E117EC11F01C0EF76E32
:1072F000360EF66E2CEC01F016D017EC11F0040EE1
:107300007A5C09E117EC11F01C0EF76E400EF66E78
:107310002CEC01F008D017EC11F01C0EF76E4A0EA1
:10732000F66E2CEC01F017EC11F0E4EC51F017ECD8
:1073300011F017EC11F00301100E4C6F000180D119
:10734000110E8F5D22E117EC11F007EC4AF017ECFB
:1073500011F017EC11F00301140E446F17EC11F04B
:10736000100E03014C5D000107E117EC11F017EC62
:1073700011F0120E8F6F06D017EC11F017EC11F010
:10738000100E8F6F7CEF30F05BD1120E8F5D47E1F6
:1073900017EC11F017EC11F090518325836F000E5C
:1073A00090BFFF0E8421846F17EC11F08451E8AE7A
:1073B00006D017EC11F017EC11F0846B836B17EC0F
:1073C00011F0800E016E0FEC00F01C0EF76E540EE3
:1073D000F66E2CEC01F017EC11F0800E016E040E2D
:1073E000056E84C018F083C017F060EC00F017EC55
:1073F00011F0200E34EC01F06D0E34EC01F0200E93
:1074000034EC01F017EC11F0E4EC51F017EC11F052
:1074100017EC11F00301120E4C6F000111D1130E85
:107420008F5D41E117EC11F09051E8AE05D017ECFB
:1074300011F017EC11F03B9417EC11F09051E8BEED
:1074400007D0905305E017EC11F017EC11F03B84D6
:1074500017EC11F0800E016E0FEC00F01C0EF76EB1
:10746000620EF66E2CEC01F017EC11F03BB40BD071
:1074700017EC11F04F0E34EC01F0460E34EC01F035
:1074800034EC01F00BD017EC11F0200E34EC01F0CD
:107490004F0E34EC01F04E0E34EC01F017EC11F00D
:1074A0001FEC52F0CDD0140E8F5D41E117EC11F0BE
:1074B0009051E8AE05D017EC11F017EC11F03B96A7
:1074C00017EC11F09051E8BE07D0905305E017EC8F
:1074D00011F017EC11F03B8617EC11F0800E016EE5
:1074E0000FEC00F01C0EF76E740EF66E2CEC01F033
:1074F00017EC11F03BB60BD017EC11F04F0E34EC3B
:1075000001F0460E34EC01F034EC01F00BD017EC36
:1075100011F0200E34EC01F04F0E34EC01F04E0E61
:1075200034EC01F017EC11F01FEC52F089D0150E7D
:107530008F5D41E117EC11F09051E8AE05D017ECEA
:1075400011F017EC11F03C9C17EC11F09051E8BED3
:1075500007D0905305E017EC11F017EC11F03C8CBC
:1075600017EC11F0800E016E0FEC00F01C0EF76EA0
:10757000860EF66E2CEC01F017EC11F03CBC0BD033
:1075800017EC11F04F0E34EC01F0460E34EC01F024
:1075900034EC01F00BD017EC11F0200E34EC01F0BC
:1075A0004F0E34EC01F04E0E34EC01F017EC11F0FC
:1075B0001FEC52F045D0160E8F5D42E117EC11F032
:1075C0009051E8AE03D017EC11F0B2D817EC11F0DF
:1075D0009051E8BE05D0905303E017EC11F0C2D9EA
:1075E00017EC11F0800E016E0FEC00F01C0EF76E20
:1075F000980EF66E2CEC01F017EC11F0200E34EC26
:1076000001F0000E34EC01F0200E34EC01F04D0ED0
:1076100034EC01F0200E34EC01F0010E34EC01F0FA
:10762000200E34EC01F034EC01F034EC01F0040EE7
:1076300034EC01F01C0EF76EAE0EF66E2CEC01F081
:1076400017EC11F017EC11F0906B17EC11F0010E24
:1076500082B4000E336E010E82B6000E331201E0CA
:10766000F6D717EC11F017EC11F0B16BB06B17EC0B
:1076700011F0010E80BC000E336E010E80BE000EB4
:10768000331217E017EC11F017EC11F0030146511B
:107690000001B027000EB12317EC11F0B051915D3D
:1076A000B151925906E317EC11F0010EBAEC01F05A
:1076B000E0D717EC11F0925303E1330E915D09E32B
:1076C00017EC11F017EC11F0190E0001915F000E8C
:1076D000925B17EC11F0000E80BC010E336E000EB1
:1076E00080BE010E3316000E82B6010E3316000E58
:1076F00082B4010E3316000E82B2010E33160FE073
:1077000017EC11F017EC11F0010E926FF40E916F5F
:1077100017EC11F003014453000101E0DCD77CEFCA
:1077200030F017EC11F017EC11F03B9817EF11F057
:1077300017EC11F017EC11F03D8A17EC11F0800EE8
:10774000016E0FEC00F01C0EF76EBA0EF66E2CEC0C
:1077500001F017EC11F0800E016E940E0FEC00F0AA
:107760001C0EF76ED00EF66E2CEC01F017EC11F03B
:1077700082A6FED717EC11F017EC11F08C6B8B6B17
:1077800017EC11F017EC11F03D9C17EC11F017EC11
:1077900011F03D8E17EC11F093988A8817EC11F0D8
:1077A000070E8C5DD00ED8B48B5DD8B05CD017ECD2
:1077B00011F04450B75D0AE14350B65D07E117ECA4
:1077C00011F017EC11F08B4B8C2B0ED017EC11F045
:1077D00017EC11F044C0B7F043C0B6F017EC11F04D
:1077E00017EC11F08C6B8B6B17EC11F0800E016EA7
:1077F000940E0FEC00F0030E056E44C01EF043C063
:107800001DF045C317F0186A14EC02F0176E10C093
:1078100018F05BEC00F017EC11F017EC48F017ECE7
:1078200011F082B21FD017EC11F093988A9817ECE0
:1078300011F017EC11F03D9A17EC11F017EC11F064
:107840000301416B17EC11F017EC11F03B9A17ECA8
:1078500011F017EC11F00301140E446F17EC11F046
:10786000000112009DD717EC11F093988A9817EC3D
:1078700011F017EC11F0446A436A17EC11F0800E16
:10788000016E940E0FEC00F01C0EF76EDA0EF66E21
:107890002CEC01F017EC11F017EC11F03D9A17ECFD
:1078A00011F017EC11F03D9E17EC11F017EC11F0F0
:1078B0003D8C17EC11F093968A8617EC11F07250FC
:1078C000435C076E73504458086E08AE36D017EC10
:1078D00011F017EC11F07250435C226E7350445853
:1078E000236E23C01EF022C01DF045C317F0186A96
:1078F00014EC02F0856F10C086F017EC11F0800ECA
:10790000016E940E0FEC00F0030E056E86C018F0A9
:1079100085C017F05BEC00F017EC11F017EC48F0A5
:1079200017EC11F0010E82B2000E336E000E3BBA5E
:10793000010E331201E001D0C2D717EC11F093967B
:107940008A9617EC11F017EC11F00301416B17EC5C
:1079500011F017EC11F00301140E446F17EC11F045
:107960000001120017EC11F017EC11F03D8A17EC32
:1079700011F0800E016E0FEC00F01C0EF76EBA0EC7
:10798000F66E2CEC01F017EC11F0800E016E940EE7
:107990000FEC00F01C0EF76ED00EF66E2CEC01F022
:1079A00017EC11F082A4FED717EC11F017EC11F0D0
:1079B0008C6B8B6B17EC11F017EC11F046C0B9F023
:1079C00045C0B8F017EC11F017EC11F03E9017EC31
:1079D00011F017EC11F03E8217EC11F0939C8A8C99
:1079E00017EC11F0070E8C5DD00ED8B48B5DD8B0BB
:1079F00058D017EC11F04650B95D0AE14550B85D1A
:107A000007E117EC11F017EC11F08B4B8C2B0ED01B
:107A100017EC11F017EC11F046C0B9F045C0B8F002
:107A200017EC11F017EC11F08C6B8B6B17EC11F05D
:107A3000800E016E940E0FEC00F0030E056E46C032
:107A40001EF045C01DF045C317F0186A14EC02F093
:107A5000176E10C018F05BEC00F017EC11F017EC8B
:107A600048F017EC11F082B21BD017EC11F017ECB4
:107A700011F03D9A17EC11F017EC11F00301426B75
:107A800017EC11F017EC11F03B9C17EC11F017EC10
:107A900011F00301140E446F17EC11F000011200F5
:107AA000A1D717EC11F0939C8A9C17EC11F017ECFE
:107AB00011F0466A456A17EC11F0800E016E940EC3
:107AC0000FEC00F01C0EF76EDA0EF66E2CEC01F0E7
:107AD00017EC11F017EC11F03D9A17EC11F017ECC0
:107AE00011F03E9217EC11F017EC11F03E8017ECFC
:107AF00011F0939A8A8A17EC11F07450455C076E66
:107B000075504658086E08AE36D017EC11F017ECD9
:107B100011F07450455C226E75504658236E23C098
:107B20001EF022C01DF045C317F0186A14EC02F0D5
:107B3000856F10C086F017EC11F0800E016E940E68
:107B40000FEC00F0030E056E86C018F085C017F02C
:107B50005BEC00F017EC11F017EC48F017EC11F0AB
:107B6000010E82B2000E336E000E3BBC010E3312CA
:107B700001E001D0C2D717EC11F0939A8A9A17EC62
:107B800011F017EC11F00301426B17EC11F017EC38
:107B900011F00301140E446F17EC11F000011200F4
:107BA00017EC11F0AF6BAE6B010EAF5D04E325E196
:107BB0002C0EAE5D22E217EC11F0010EBAEC01F0D2
:107BC00017EC11F0AFC010F0AEC00FF0146A0A0E3F
:107BD000136EFDEC01F018C008F017C007F0085054
:107BE0000710000104E117EC11F017EC48F017EC56
:107BF00011F0AE2B000EAF23D7E317EF11F017EC07
:107C000011F017EC11F09E6B17EC11F0B2EC49F08B
:107C100017EC11F017EC11F001EEA1F012EE18F0D4
:107C2000030EB2EC02F0EF6A17EC11F01C0EF76EC7
:107C3000E20EF66E01EEA1F0D0EC02F0336E000E13
:107C40003AB0010E3312000E3AB2010E331209E0BF
:107C500017EC11F017EC11F000EEE6F0EF6A17EFF9
:107C600011F017EC11F017EC11F0010E9D6F17ECED
:107C700011F017EC11F09A6B17EC11F000EEE6F032
:107C80009D51EB50076E2A0E075C0EE017EC11F0C9
:107C900017EC11F000EEE6F09D51EB50076E9A1BC9
:107CA00017EC11F09D2BEAD717EC11F09D2B17EC78
:107CB00011F017EC11F000EEE6F09D51EB50146E50
:107CC000FC0EF66E1C0EF76EF86A1368132A13503A
:107CD0000F0806E30900F550145CF8E113C09BF0AF
:107CE00017EC11F017EC11F09B39F00B9C6F17ECAF
:107CF00011F09D2B17EC11F017EC11F000EEE6F0EF
:107D00009D51EB50146E0C0EF66E1D0EF76EF86A58
:107D10001368132A13500F0806E30900F550145C8A
:107D2000F8E113C09BF017EC11F017EC11F09C5127
:107D30009B2717EC11F09A519B5D02E017EF11F0B1
:107D400017EC11F017EC11F09E6B17EC11F0ACEC86
:107D500049F017EC11F002011C51076E2E0E075C62
:107D6000000102E017EF11F017EC11F017EC11F021
:107D700001EEA1F012EE18F0020EE6CFEEFFE82EB3
:107D8000FCD7EF6A17EC11F017EC11F001EEA1F03F
:107D900016EC00F00301136F17EC11F017EC11F063
:107DA00001EEA1F012EE18F0030EF36E020EA9EC34
:107DB00002F0EF6A17EC11F017EC11F001EEA1F0F0
:107DC00016EC00F01AC02DF019C02CF018C02BF0E2
:107DD00017C02AF08EEC08F02DC017F32CC016F354
:107DE0002BC015F32AC014F317EC11F0010E030198
:107DF0001353D8A4000E336E2D6A2C6A2B6A2A6A9C
:107E000017C331F016C330F015C32FF014C32EF092
:107E100026EC06F03316000105E017EC11F017EC24
:107E200011F03E8617EC11F0B40E0301135D010E44
:107E3000D8A4000E336E2D6A2C6A2B6A2A6A17C3E7
:107E400031F016C330F015C32FF014C32EF026EC1A
:107E500006F03316000105E017EC11F017EC11F0F5
:107E60003E8617EC11F017EC11F001EEA1F012EEC6
:107E700018F0060EF36E020EA9EC02F0EF6A17EC92
:107E800011F017EC11F001EEA1F016EC00F01AC0A1
:107E90002DF019C02CF018C02BF017C02AF08EEC72
:107EA00008F02DC05CF32CC05BF32BC05AF32AC042
:107EB00059F317EC11F017EC11F0316A306A480EE3
:107EC0002F6E850E2E6E5CC32DF05BC32CF05AC353
:107ED0002BF059C32AF07DEC07F02DC025F02CC003
:107EE00024F02BC023F02AC022F017C331F016C3B0
:107EF00030F015C32FF014C32EF025C02DF024C090
:107F00002CF023C02BF022C02AF0EFEC06F02DC09D
:107F100017F32CC016F32BC015F32AC014F317EC7B
:107F200011F017EC11F0316A306A700E2F6E840E6A
:107F30002E6E17C32DF016C32CF015C32BF014C3EF
:107F40002AF07DEC07F02DC025F02CC024F02BC0CA
:107F500023F02AC022F0030113518AEC08F025C057
:107F600031F024C030F023C02FF022C02EF0EFEC0F
:107F700006F02DC01BF32CC01AF32BC019F32AC036
:107F800018F317EC11F02D6A2C6A340E2B6E850E47
:107F90002A6E1BC331F01AC330F019C32FF018C377
:107FA0002EF06BEC06F00108000102E017EF11F073
:107FB00017EC11F017EC11F09E6B17EC11F0A9EC17
:107FC00049F017EC11F002EE18F0EECFF3FFEFCF0F
:107FD000F4FFF350530AF41006E117EC11F017EC1C
:107FE00011F00301197F000117EC11F017EC11F0EB
:107FF0009E6B17EC11F0A6EC49F017EC11F00201A2
:108000001D51076E2E0E075C000102E017EF11F004
:1080100017EC11F017EC11F001EEA1F012EE18F0D0
:10802000030EE6CFEEFFE82EFCD7EF6A17EC11F057
:1080300017EC11F001EEA1F016EC00F00301136F44
:1080400017EC11F017EC11F001EEA1F012EE18F0A0
:10805000040EF36E020EA9EC02F0EF6A17EC11F0B9
:1080600017EC11F001EEA1F016EC00F01AC02DF0A3
:1080700019C02CF018C02BF017C02AF08EEC08F0B5
:108080002DC017F32CC016F32BC015F32AC014F320
:1080900017EC11F0010E03011353D8A4000E336E38
:1080A0002D6A2C6A2B6A2A6A17C331F016C330F086
:1080B00015C32FF014C32EF026EC06F03316000E75
:1080C0003EB6010E3316000109E017EC11F017EC73
:1080D00011F000EEE6F0EF6A17EF11F017EC11F077
:1080E00017EC11F001EEA1F012EE18F0070EF36E8E
:1080F000020EA9EC02F0EF6A17EC11F017EC11F088
:1081000001EEA1F016EC00F01AC02DF019C02CF011
:1081100018C02BF017C02AF08EEC08F02DC05CF3CD
:108120002CC05BF32BC05AF32AC059F317EC11F0A3
:1081300017EC11F0316A306A480E2F6E850E2E6EE4
:108140005CC32DF05BC32CF05AC32BF059C32AF04B
:108150007DEC07F02DC025F02CC024F02BC023F0BF
:108160002AC022F017C331F016C330F015C32FF028
:1081700014C32EF025C02DF024C02CF023C02BF00A
:1081800022C02AF0EFEC06F02DC017F32CC016F336
:108190002BC015F32AC014F317EC11F017EC11F0F3
:1081A000316A306A700E2F6E840E2E6E17C32DF05A
:1081B00016C32CF015C32BF014C32AF07DEC07F086
:1081C0002DC025F02CC024F02BC023F02AC022F0B3
:1081D000030113518AEC08F025C031F024C030F0BF
:1081E00023C02FF022C02EF0EFEC06F02DC01FF3BD
:1081F0002CC01EF32BC01DF32AC01CF317EC11F08A
:108200002D6A2C6A340E2B6E860E2A6E1FC331F037
:108210001EC330F01DC32FF01CC32EF033EC06F04C
:108220000108000102E017EF11F017EC11F017EC54
:1082300011F09E6B17EC11F0A3EC49F017EC11F064
:1082400002EE18F0EECFF3FFEFCFF4FFF350570A32
:10825000F41006E117EC11F017EC11F003011D7F8B
:10826000000117EC11F017EC11F09E6B17EC11F0F8
:1082700097EC49F017EC11F017EC11F002EE18F042
:1082800016EC00F00301286F18C029F317EC11F069
:1082900017EC11F001EEA1F012EE18F0010EB2ECA5
:1082A00002F0EF6A17EC11F00101A151076E350ED3
:1082B000075C000105E317EC11F00301284B292BA3
:1082C000000117EC11F09C0E0301295D00010AE387
:1082D00005E1410E0301285D000104E317EC11F0F4
:1082E0000001120017EC11F017EC11F0D00E2D6EFA
:1082F0000F0E2C6E490E2B6E800E2A6E1BC331F0B2
:108300001AC330F019C32FF018C32EF0E3EC07F0B6
:108310002DC025F02CC024F02BC023F02AC022F061
:10832000316A306A340E2F6E860E2E6E25C02DF007
:1083300024C02CF023C02BF022C02AF07DEC07F0E3
:108340002DC05CF32CC05BF32BC05AF32AC059F349
:1083500017EC11F017EC11F05CC32DF05BC32CF09F
:108360005AC32BF059C32AF00CEC04F02DC0A7F02F
:108370002CC0A6F02BC0A5F02AC0A4F017EC11F079
:1083800017EC11F01FC325F01EC324F01DC323F00A
:108390001CC322F025C02DF024C02CF023C02BF0EC
:1083A00022C02AF031C331F030C330F02FC32FF098
:1083B0002EC32EF0EDEC06F02DC025F02CC024F0DD
:1083C0002BC023F02AC022F025C031F024C030F0A9
:1083D00023C02FF022C02EF0A7C02DF0A6C02CF095
:1083E000A5C02BF0A4C02AF0E3EC07F02DC025F0C7
:1083F0002CC024F02BC023F02AC022F09A0E2D6E40
:10840000990E2C6E5E0E2B6E850E2A6E25C031F0F5
:1084100024C030F023C02FF022C02EF0E3EC07F090
:108420002DC03BF32CC03AF32BC039F32AC038F3EC
:1084300017EC11F017EC11F01BC32DF01AC32CF040
:1084400019C32BF018C32AF02DC331F02CC330F020
:108450002BC32FF02AC32EF0EDEC06F02DC025F033
:108460002CC024F02BC023F02AC022F09A0E2D6ECF
:10847000990E2C6E5E0E2B6E850E2A6E25C031F085
:1084800024C030F023C02FF022C02EF0E3EC07F020
:108490002DC037F32CC036F32BC035F32AC034F38C
:1084A00017EC11F017EC11F037C331F036C330F090
:1084B00035C32FF034C32EF037C32DF036C32CF064
:1084C00035C32BF034C32AF0E3EC07F031EC08F0AD
:1084D00003015D6F2BC05EF32CC05FF32DC060F312
:1084E00017EC11F017EC11F03BC331F03AC330F048
:1084F00039C32FF038C32EF03BC32DF03AC32CF014
:1085000039C32BF038C32AF0E3EC07F031EC08F064
:108510000301616F2BC062F32CC063F32DC064F3C1
:1085200017EC11F017EC11F0030161515D254D6F4F
:1085300062515E214E6F63515F214F6F6451602124
:10854000506F17EC11F017EC11F050C32DF04FC322
:108550002CF04EC32BF04DC32AF090EC08F07BECCE
:1085600005F02DC070F32CC06FF32BC06EF32AC042
:108570006DF317EC11F017EC11F0316A306A7A0ED6
:108580002F6E880E2E6E33C32BF032C32AF084EC8C
:1085900008F07DEC07F02DC025F02CC024F02BC096
:1085A00023F02AC022F02D6A500E2C6E470E2B6E3F
:1085B0008B0E2A6E25C031F024C030F023C02FF07E
:1085C00022C02EF0EFEC06F02DC06CF32CC06BF344
:1085D0002BC06AF32AC069F317EC11F017EC11F005
:1085E0006CC331F06BC330F06AC32FF069C32EF057
:1085F0006CC32DF06BC32CF06AC32BF069C32AF057
:10860000E3EC07F031EC08F003015D6F2BC05EF383
:108610002CC05FF32DC060F317EC11F017EC11F0D4
:1086200070C331F06FC330F06EC32FF06DC32EF006
:1086300070C32DF06FC32CF06EC32BF06DC32AF006
:10864000E3EC07F031EC08F00301616F2BC062F33B
:108650002CC063F32DC064F317EC11F017EC11F08C
:10866000030161515D254D6F62515E214E6F635173
:108670005F214F6F64516021506F17EC11F017ECC0
:1086800011F050C32DF04FC32CF04EC32BF04DC34F
:108690002AF090EC08F07BEC05F02DC0A7F02CC080
:1086A000A6F02BC0A5F02AC0A4F017EC11F017EC2F
:1086B00011F0A7C025F0A6C024F0A5C023F0A4C0E7
:1086C00022F025C02DF024C02CF023C02BF022C0B6
:1086D0002AF06CC331F06BC330F06AC32FF069C36A
:1086E0002EF0EDEC06F02DC025F02CC024F02BC0B0
:1086F00023F02AC022F02D6A2C6A7A0E2B6E880E87
:108700002A6E25C031F024C030F023C02FF022C0E3
:108710002EF0E3EC07F02DC025F02CC024F02BC088
:1087200023F02AC022F033C32BF032C32AF084ECAA
:1087300008F025C031F024C030F023C02FF022C053
:108740002EF0EFEC06F031EC08F003015D6F2BC06A
:108750005EF32CC05FF32DC060F317EC11F0030142
:1087600060530001D8A4B3D003015F530001D8A423
:10877000AED003015E51295D0001D8A0A8D006E16A
:10878000030128515D5D0001D8B0A1D017EC11F0B4
:1087900017EC11F003015D51285D616F5E5129599D
:1087A000626F000E5F55636F000E6055646F17ECCB
:1087B00011F017EC11F070C331F06FC330F06EC3DD
:1087C0002FF06DC32EF064C32DF063C32CF062C391
:1087D0002BF061C32AF08EEC08F07DEC07F02DC081
:1087E00025F02CC024F02BC023F02AC022F0316ADF
:1087F000306A7A0E2F6E880E2E6E25C02DF024C0A2
:108800002CF023C02BF022C02AF07DEC07F02DC005
:10881000A7F02CC0A6F02BC0A5F02AC0A4F017EC3E
:1088200011F017EC11F0A7C02DF0A6C02CF0A5C0D8
:108830002BF0A4C02AF0DAEC02F02DC05CF32CC0BF
:108840005BF32BC05AF32AC059F317EC11F017EC65
:1088500011F05CC327F35BC326F35AC325F359C356
:1088600024F317EC11F017EC11F02D6A2C6A340E7A
:108870002B6E860E2A6E5CC331F05BC330F05AC398
:108880002FF059C32EF0E3EC07F02DC025F02CC0DB
:1088900024F02BC023F02AC022F0D00E316E0F0E30
:1088A000306E490E2F6E800E2E6E25C02DF024C026
:1088B0002CF023C02BF022C02AF07DEC07F0E3EC73
:1088C00006F00301716F2BC072F3000107D017ECA3
:1088D00011F017EC11F00301726B716B000117ECD2
:1088E00011F00301725304E15B0E715D00010AE3B4
:1088F00017EC11F017EC11F0426A416A17EC11F015
:108900000001120017EC11F017EC11F003014551B2
:108910007103F3CF41F0F4CF42F07203F3504226DB
:1089200017EC11F0000142AE08D017EC11F017EC73
:1089300011F0426A416A17EF11F017EC11F017ECD1
:1089400011F042C02BF041C02AF084EC08F02DC099
:1089500027F32CC026F32BC025F32AC024F317ECF1
:1089600011F04150B45D0F6E4250B559106E91EC4C
:1089700002F0076E10C008F003014551050DF3CF5A
:108980000BF0F4CF0CF00D6A0E6A0E52000120E1DC
:108990000D521EE10C50085C1BE303E107500B5C19
:1089A00017E217EC11F00001A02B17EC11F0030EE9
:1089B000A05D0DE317EC11F017EC11F042C0B5F01B
:1089C00041C0B4F017EC11F017EC11F0A06B05D01A
:1089D00017EC11F017EC11F0A06B17EC11F017EC7D
:1089E00011F03BC32DF03AC32CF039C32BF038C340
:1089F0002AF037C331F036C330F035C32FF034C31B
:108A00002EF07DEC07F02DC0A7F02CC0A6F02BC0F7
:108A1000A5F02AC0A4F017EC11F017EC11F0A7C0D4
:108A20002DF0A6C02CF0A5C02BF0A4C02AF0DAECE3
:108A300002F02DC05CF32CC05BF32BC05AF32AC0AC
:108A400059F317EC11F017EC11F02D6A2C6A340E63
:108A50002B6E860E2A6E5CC331F05BC330F05AC3B6
:108A60002FF059C32EF0E3EC07F02DC025F02CC0F9
:108A700024F02BC023F02AC022F0D00E316E0F0E4E
:108A8000306E490E2F6E800E2E6E25C02DF024C044
:108A90002CF023C02BF022C02AF07DEC07F02DC073
:108AA0005CF32CC05BF32BC05AF32AC059F317ECCC
:108AB00011F017EC11F05CC323F35BC322F35AC32C
:108AC00021F359C320F317EC11F017EC11F05CC33C
:108AD0002DF05BC32CF05AC32BF059C32AF0E3EC02
:108AE00006F00301716F2BC072F317EC11F037C35E
:108AF0002DF036C32CF035C32BF034C32AF0316A85
:108B0000306A2F6A2E6A6BEC06F0336E3BC32DF091
:108B10003AC32CF039C32BF038C32AF0316A306ADB
:108B20002F6A2E6AA7EC06F03316000125E017EC39
:108B300011F017EC11F0680E03017127010E72237A
:108B400017EC11F017EC11F02D6A2C6A340E2B6E15
:108B5000870E2A6E23C331F022C330F021C32FF0D9
:108B600020C32EF0EFEC06F02DC023F32CC022F32F
:108B70002BC021F32AC020F3000117EC11F00301F0
:108B800035510001E8AE25D017EC11F017EC11F0CB
:108B9000B40E03017127000E722317EC11F017ECCD
:108BA00011F02D6A2C6A340E2B6E860E2A6E23C3AA
:108BB00031F022C330F021C32FF020C32EF0EFECB0
:108BC00006F02DC023F32CC022F32BC021F32AC0C2
:108BD00020F3000117EC11F017EC11F072C340F014
:108BE00071C33FF017EC11F0030171510001B25D48
:108BF0000F6E030172510001B359106E91EC02F037
:108C0000076E10C008F0085203E1060E075C17E378
:108C100017EC11F000019F2B17EC11F0030E9F5D74
:108C20000DE317EC11F017EC11F072C3B3F071C340
:108C3000B2F017EC11F017EC11F09F6B05D017ECA8
:108C400011F017EC11F09F6B17EC11F017EC11F00D
:108C500000EEE6F0EF6A17EC11F09F5302E1000E10
:108C600001D0010E336EA05302E1000E01D0010EBF
:108C7000331202E017EF11F017EC11F017EC11F0BE
:108C800072C3B3F071C3B2F017EC11F017EC11F02E
:108C900042C0B5F041C0B4F017EC11F01E0E030154
:108CA0004B5D000102E217EF11F017EC11F017EC29
:108CB00011F0030145517103F3CF3FF0F4CF40F0C1
:108CC0007203F350402617EC11F000016BD817EC3B
:108CD00011F03CBA50D017EC11F06C50435C076EA9
:108CE0006D504458086E6DBEFF0E000E096A44BEFA
:108CF00009686DBEFF0E095A0A6A09BE0A68075064
:108D00005B180BE108505C1808E109505CBE0928AB
:108D100004E10A505CBE0A2805E017EC11F017ECDC
:108D200011F03A80000117EC11F06E50455C076EAF
:108D30006F504658086E6FBEFF0E000E096A46BEA1
:108D400009686FBEFF0E095A0A6A09BE0A68075011
:108D500041180BE10850421808E1095042BE0928A9
:108D600004E10A5042BE0A2805E017EC11F017ECA6
:108D700011F03A82000117EC11F017EC11F0030129
:108D80004B6B17EC11F0000E3AB0010E336E000E73
:108D90003AB2010E3312000103E017EC11F0FBD8D8
:108DA00017EF11F017EC11F09351E8A617D017EC5C
:108DB00011F017EC11F0BA513F5C5B6EBB5140589B
:108DC0005C6E17EC11F05CAE08D017EC11F017ECEC
:108DD00011F0BC515B26BD515C2208D017EC11F09C
:108DE00017EC11F040C05CF03FC05BF017EC11F0E5
:108DF00017EC11F06C505B266D505C2217EC11F0F3
:108E00009335D8A0C6D017EC11F071BE14D0120E55
:108E1000715C11E303E15D0E705C0DE317EC11F082
:108E200017EC11F0AA6A0C0EA96EB3EC01F0706E8B
:108E3000B3EC01F0716E000117EC11F0BC515B2432
:108E4000076EBD515C20086E7050075C7150085869
:108E500008507118D8B0800A02E7000E01D0010E48
:108E6000336E030145510E0DF3CF22F0F4CF23F002
:108E7000246A2326000E242245AF04D00E0E235E62
:108E8000010E245A0001256A24BE25066C502224B6
:108E9000076E6D502320086E000E6DBEFF0E24205D
:108EA000096E000E6DBEFF0E25200A6E43C00FF046
:108EB00044C010F0000E10BEFF0E116E126E0F5067
:108EC000075C105008581150095812500A58125097
:108ED0000A18D8B0800A02E7000E01D0010E33163E
:108EE00008E017EC11F017EC11F0BC515B26BD51F6
:108EF0005C2217EC11F06C50C425076E6D50C52133
:108F0000086E000E08BEFF0E096E0A6E43C00FF019
:108F100044C010F0000E10BEFF0E116E126E07500E
:108F20000F5C08501058095011580A5012580A5036
:108F30001218D8B0800A02E7000E01D0010E336E7D
:108F4000BC515B5C076EBD515C58086E000E03019E
:108F500045BFFF0E085C07E008504519D8B0800AED
:108F6000800B07E008D0000107500301455D0001B8
:108F700002E3000E01D0010E331600010AE017ECE7
:108F800011F017EC11F0BC515B5C5B6EBD515C588D
:108F90005C6E17EF11F017EC11F0000E81B6010EA8
:108FA000336E000E81B8010E3312000E81BA010E2D
:108FB0003312000E81BC010E3312010E93BB000E62
:108FC000331202E017EF11F017EC11F09351E8A8FB
:108FD00020D017EC11F0986B7E0E985D16E217EC1E
:108FE00011F0939E8A8E17EC11F0C80EC7EC01F0B9
:108FF00017EC11F0939E8A9E17EC11F0C80EC7EC87
:1090000001F017EC11F0982BE7E317EC11F0938EB9
:109010000CD017EC11F0939E8A8E17EC11F0320EE3
:10902000BAEC01F017EC11F0938E17EF11F017EC7A
:1090300011F0E86A3CBE010F83BC0108D8A4010E00
:10904000336EE86A3DB0010F83BE0108D8A4010E5B
:109050003312D8B48ED017EC11F0020EBAEC01F036
:1090600017EC11F0E86A3CBE010F83BC0108D8A4DC
:10907000010E336EE86A3DB0010F83BE0108D8A42B
:10908000010E3312D8B475D017EC11F0020EBAEC01
:1090900001F017EC11F0E86A3CBE010F83BC010837
:1090A0002FE017EC11F017EC11F03C8E83AC3C9ED6
:1090B00017EC11F03DAC04D017EC11F0434A442AF0
:1090C00017EC11F03DAE06D017EC11F0010E435E27
:1090D000000E445A17EC11F0E86A81B6010F81B80E
:1090E000010808E117EC11F093968A9617EC11F03D
:1090F00093988A9817EC11F017EC11F00301416B6B
:10910000000117EC11F0E86A3DB0010F83BE0108C1
:109110002FE017EC11F017EC11F03D8083AE3D907D
:1091200017EC11F03EA004D017EC11F0454A462A86
:1091300017EC11F03EA206D017EC11F0010E455EBF
:10914000000E465A17EC11F0E86A81BC010F81BA93
:10915000010808E117EC11F0939A8A9A17EC11F0C4
:10916000939C8A9C17EC11F017EC11F00301426BF1
:10917000000117EF11F0000E9EBA010E336E010EC2
:1091800082B0000E3316D8B454D0AECFA1F0610E29
:10919000A15D000ED8B0010E336E7B0EA15D02E31F
:1091A000000E01D0010E331601E0A19B933103E3C1
:1091B000A1518EEC01F09E9A0A0EA15D17E001EE1E
:1091C00037F0EE50FEE1ED52A1C0EEFFEF6A4E0E19
:1091D0000301405D000104E20301402B000105D0C2
:1091E0000301406B01EE37F0EF6A0001240EA15D30
:1091F00008E101EE37F0EF6A01EE37F0A1C0EEFFB3
:10920000EF6A0D0EA15D15E13D880301406B000181
:10921000D20EA36F00EEE6F011EE37F0500EE752DB
:1092200004E0E6CFEEFFE82EFAD7EF6A01EE37F062
:10923000EF6A9EA47AD09E94972B0F0E975DD8A0CC
:1092400074D0976B000E3EB4010E010AD8B43E9460
:10925000D8A43E84000E3BBC010E336E000E3BBA18
:10926000010E331217E0A22B0D0EA25D13E33B9CFF
:109270003B9A0301416B426B0001A26B44C050F06A
:1092800043C04FF046C052F045C051F03A903A9872
:109290003A923A9AFA0E03014B5D000102E2030191
:1092A0004B2B03014453000102E00301440700017A
:1092B0003DBA33D0000E81B6010E336E000E81B878
:1092C000010E331202E00301412B0001000E81BAAE
:1092D000010E336E000E81BC010E331202E0030159
:1092E000422B050E0301415D000109E33B8A93987F
:1092F0008A9893968A9644C050F043C04FF0050E6A
:109300000301425D000109E33B8C939A8A9A939C86
:109310008A9C46C052F045C051F0BE0E0301735DF9
:10932000000102E20301732B00011100000117ECA0
:1093300011F051D817EC11F04ED817EC11F04BD8B2
:1093400017EC11F048D817EC11F045D817EC11F0D4
:1093500042D817EC11F03FD817EC11F03CD817ECBD
:1093600011F039D817EC11F017EC11F09D6B17ECD8
:1093700011F000EEE6F09E51EB50076E2C0E075CEC
:109380001DE017EC11F017EC11F000EEE6F09E5125
:10939000EBCF07F002EE18F09D51E926000EEA220D
:1093A00007C0EFFF17EC11F04E0E9D5D03E217ECC6
:1093B00011F09D2B17EC11F09E2BDBD717EC11F061
:1093C00017EC11F002EE18F09D51E926000EEA228A
:1093D000EF6A17EF11F017EC11F000EEE6F09E5176
:1093E000EB50076E2C0E075CD8A4010E336E500EA6
:1093F0009E5D010ED8B0000E331604E017EC11F09C
:109400009E2BEBD717EC11F09E2B17EF11F017ECFA
:1094100011F017EC11F00301040E4A6F17EC11F074
:109420000001010E82B6000E336E010E82B4000EF2
:109430003312010E80BC000E3312010E80BE000EEE
:10944000331201E0EDD717EC11F082A256EF4FF086
:1094500017EC11F0ACEC4FF017EC11F080BC11D20E
:1094600017EC11F0040E03014A5D010ED8A4000EA2
:10947000336E2DC32DF02CC32CF02BC32BF02AC33D
:109480002AF0316A306A200E2F6E820E2E6E33EC77
:1094900006F0331600011CE017EC11F017EC11F088
:1094A000316A306A200E2F6E820E2E6E2DC32DF083
:1094B0002CC32CF02BC32BF02AC32AF0EDEC06F0C2
:1094C0002DC02DF32CC02CF32BC02BF32AC02AF374
:1094D00017EC11F0050E03014A5D010ED8A4000E31
:1094E000336E2DC32DF02CC32CF02BC32BF02AC3CD
:1094F0002AF0316A306A2F6A7F0E2E6E33EC06F046
:10950000331600011BE017EC11F017EC11F0316A73
:10951000306A2F6A7F0E2E6E2DC32DF02CC32CF0D7
:109520002BC32BF02AC32AF0EDEC06F02DC02DF34F
:109530002CC02CF32BC02BF32AC02AF317EC11F00C
:10954000070E03014A5D010ED8A4000E336E2DC331
:109550002DF02CC32CF02BC32BF02AC32AF0CD0EF8
:10956000316ECC0E306E4C0E2F6E7B0E2E6E33ECA9
:1095700006F0331600011EE017EC11F017EC11F0A5
:10958000CD0E316ECC0E306E4C0E2F6E7B0E2E6ECD
:109590002DC32DF02CC32CF02BC32BF02AC32AF0A3
:1095A000EDEC06F02DC02DF32CC02CF32BC02BF3CB
:1095B0002AC02AF317EC11F0080E03014A5D010ED0
:1095C000D8A4000E336E2DC32DF02CC32CF02BC36A
:1095D0002BF02AC32AF00A0E316ED70E306E230EFE
:1095E0002F6E780E2E6E33EC06F0331600011EE05F
:1095F00017EC11F017EC11F00A0E316ED70E306E29
:10960000230E2F6E780E2E6E2DC32DF02CC32CF052
:109610002BC32BF02AC32AF0EDEC06F02DC02DF35E
:109620002CC02CF32BC02BF32AC02AF317EC11F01B
:109630000E0E03014A5D010ED8A4000E336E31C335
:109640002DF030C32CF02FC32BF02EC32AF0316A3B
:10965000306A480E2F6E850E2E6E33EC06F03316F0
:1096600000011CE017EC11F017EC11F0316A306AC0
:10967000480E2F6E850E2E6E31C32DF030C32CF0A8
:109680002FC32BF02EC32AF0EDEC06F02DC031F3E2
:109690002CC030F32BC02FF32AC02EF317EC11F09F
:1096A0000F0E03014A5D010ED8A4000E336E31C3C4
:1096B0002DF030C32CF02FC32BF02EC32AF0316ACB
:1096C000306A200E2F6E820E2E6E33EC06F03316AB
:1096D00000011CE017EC11F017EC11F0316A306A50
:1096E000200E2F6E820E2E6E31C32DF030C32CF063
:1096F0002FC32BF02EC32AF0EDEC06F02DC031F372
:109700002CC030F32BC02FF32AC02EF317EC11F02E
:10971000100E03014A5D010ED8A4000E336E31C352
:109720002DF030C32CF02FC32BF02EC32AF0316A5A
:10973000306A2F6A7F0E2E6E33EC06F0331600016E
:109740001BE017EC11F017EC11F0316A306A2F6A48
:109750007F0E2E6E31C32DF030C32CF02FC32BF0B3
:109760002EC32AF0EDEC06F02DC031F32CC030F3FF
:109770002BC02FF32AC02EF317EC11F0120E0301A9
:109780004A5D010ED8A4000E336E31C32DF030C3F4
:109790002CF02FC32BF02EC32AF0CD0E316ECC0E41
:1097A000306E4C0E2F6E7B0E2E6E33EC06F03316A1
:1097B00000011EE017EC11F017EC11F0CD0E316E28
:1097C000CC0E306E4C0E2F6E7B0E2E6E31C32DF0F4
:1097D00030C32CF02FC32BF02EC32AF0EDEC06F093
:1097E0002DC031F32CC030F32BC02FF32AC02EF341
:1097F00017EC11F0130E03014A5D010ED8A4000E00
:10980000336E31C32DF030C32CF02FC32BF02EC399
:109810002AF00A0E316ED70E306E230E2F6E780EA0
:109820002E6E33EC06F0331600011EE017EC11F03B
:1098300017EC11F00A0E316ED70E306E230E2F6E1C
:10984000780E2E6E31C32DF030C32CF02FC32BF0C9
:109850002EC32AF0EDEC06F02DC031F32CC030F30E
:109860002BC02FF32AC02EF317EC11F017EC11F0D8
:109870003E9417EC11F0ACEC4FF017EC11F080AC0B
:10988000FED717EC11F080BEC4EF4EF017EC11F0CC
:10989000040E03014A5D00013DE117EC11F02DC3F8
:1098A0002DF02CC32CF02BC32BF02AC32AF0316AE5
:1098B000306A200E2F6E850E2E6E6BEC06F00108BE
:1098C0001DE017EC11F017EC11F02D6A2C6A200E38
:1098D0002B6E820E2A6E2DC331F02CC330F02BC3B9
:1098E0002FF02AC32EF0EFEC06F02DC02DF32CC084
:1098F0002CF32BC02BF32AC02AF30BD017EC11F05A
:1099000017EC11F003012D6B2C6B340E2B6F850EB1
:109910002A6F000117EC11F0050E03014A5D0001EA
:109920003CE117EC11F02DC32DF02CC32CF02BC310
:109930002BF02AC32AF0316A306A320E2F6E850E60
:109940002E6E6BEC06F001081CE017EC11F017EC22
:1099500011F02D6A2C6A2B6A7F0E2A6E2DC331F00E
:109960002CC330F02BC32FF02AC32EF0EFEC06F0FF
:109970002DC02DF32CC02CF32BC02BF32AC02AF3BF
:109980000BD017EC11F017EC11F003012D6B2C6BC1
:10999000340E2B6F850E2A6F000117EC11F0070EA5
:1099A00003014A5D000141E117EC11F02DC32DF0D8
:1099B0002CC32CF02BC32BF02AC32AF0CD0E316E12
:1099C000CC0E306E330E2F6E850E2E6E6BEC06F0C5
:1099D00001081FE017EC11F017EC11F0CD0E2D6E01
:1099E000CC0E2C6E4C0E2B6E7B0E2A6E2DC331F0DE
:1099F0002CC330F02BC32FF02AC32EF0EFEC06F06F
:109A00002DC02DF32CC02CF32BC02BF32AC02AF32E
:109A10000BD017EC11F017EC11F003012D6B2C6B30
:109A2000340E2B6F850E2A6F000117EC11F0080E13
:109A300003014A5D000141E117EC11F02DC32DF047
:109A40002CC32CF02BC32BF02AC32AF0E10E316E6D
:109A5000FA0E306E330E2F6E850E2E6E6BEC06F006
:109A600001081FE017EC11F017EC11F00A0E2D6E33
:109A7000D70E2C6E230E2B6E780E2A6E2DC331F06E
:109A80002CC330F02BC32FF02AC32EF0EFEC06F0DE
:109A90002DC02DF32CC02CF32BC02BF32AC02AF39E
:109AA0000BD017EC11F017EC11F003012D6B2C6BA0
:109AB000340E2B6F850E2A6F000117EC11F00E0E7D
:109AC00003014A5D00013DE117EC11F031C32DF0B7
:109AD00030C32CF02FC32BF02EC32AF0316A306A2A
:109AE000200E2F6E850E2E6E6BEC06F001081DE029
:109AF00017EC11F017EC11F02D6A2C6A480E2B6E42
:109B0000850E2A6E31C331F030C330F02FC32FF0F1
:109B10002EC32EF0EFEC06F02DC031F32CC030F345
:109B20002BC02FF32AC02EF30BD017EC11F017EC3B
:109B300011F00301316B306B340E2F6F860E2E6FD8
:109B4000000117EC11F00F0E03014A5D00013DE129
:109B500017EC11F031C32DF030C32CF02FC32BF0D4
:109B60002EC32AF0316A306A2A0E2F6E860E2E6EB0
:109B70006BEC06F001081DE017EC11F017EC11F08A
:109B80002D6A2C6A200E2B6E820E2A6E31C331F0A4
:109B900030C330F02FC32FF02EC32EF0EFEC06F0C1
:109BA0002DC031F32CC030F32BC02FF32AC02EF37D
:109BB0000BD017EC11F017EC11F00301316B306B87
:109BC000340E2F6F860E2E6F000117EC11F0100E61
:109BD00003014A5D00013CE117EC11F031C32DF0A7
:109BE00030C32CF02FC32BF02EC32AF0316A306A19
:109BF000330E2F6E860E2E6E6BEC06F001081CE005
:109C000017EC11F017EC11F02D6A2C6A2B6A7F0EFD
:109C10002A6E31C331F030C330F02FC32FF02EC382
:109C20002EF0EFEC06F02DC031F32CC030F32BC03A
:109C30002FF32AC02EF30BD017EC11F017EC11F014
:109C40000301316B306B340E2F6F860E2E6F0001C7
:109C500017EC11F0120E03014A5D000141E117EC0F
:109C600011F031C32DF030C32CF02FC32BF02EC3D5
:109C70002AF0660E316EE60E306E330E2F6E860EB3
:109C80002E6E6BEC06F001081FE017EC11F017ECDC
:109C900011F0CD0E2D6ECC0E2C6E4C0E2B6E7B0E5D
:109CA0002A6E31C331F030C330F02FC32FF02EC3F2
:109CB0002EF0EFEC06F02DC031F32CC030F32BC0AA
:109CC0002FF32AC02EF30BD017EC11F017EC11F084
:109CD0000301316B306B340E2F6F860E2E6F000137
:109CE00017EC11F0130E03014A5D000141E117EC7E
:109CF00011F031C32DF030C32CF02FC32BF02EC345
:109D00002AF0710E316EFD0E306E330E2F6E860E00
:109D10002E6E6BEC06F001081FE017EC11F017EC4B
:109D200011F00A0E2D6ED70E2C6E230E2B6E780EB0
:109D30002A6E31C331F030C330F02FC32FF02EC361
:109D40002EF0EFEC06F02DC031F32CC030F32BC019
:109D50002FF32AC02EF30BD017EC11F017EC11F0F3
:109D60000301316B306B340E2F6F860E2E6F0001A6
:109D700017EC11F017EC11F03E9417EC11F0ECD841
:109D800017EC11F080AEFED717EC11F082B644D07C
:109D900017EC11F003014A0717EC11F00D0E030147
:109DA0004A5D000107E117EC11F017EC11F0030117
:109DB000080E4A6F000117EC11F0030E03014A5D13
:109DC000000107E117EC11F017EC11F00301040E8C
:109DD0004A6F000117EC11F0110E03014A5D010EEC
:109DE000D8A4000E336E060E4A5D010ED8A4000EF4
:109DF0003312000104E017EC11F003014A070001DF
:109E000017EC11F017EC11F03E8417EC11F0A4D808
:109E100017EC11F082A6FED717EC11F082B444D0F3
:109E200017EC11F003014A2B17EC11F0140E03018B
:109E30004A5D000107E117EC11F017EC11F0030186
:109E4000130E4A6F000117EC11F0090E03014A5D71
:109E5000000107E117EC11F017EC11F003010E0EF1
:109E60004A6F000117EC11F0110E03014A5D010E5B
:109E7000D8A4000E336E060E4A5D010ED8A4000E63
:109E80003312000104E017EC11F003014A2B00012A
:109E900017EC11F017EC11F03E8417EC11F05CD8C0
:109EA00017EC11F082A4FED725EF4AF017EC11F061
:109EB00003012A517B5C0AE12B517C5C07E12C51A8
:109EC0007D5C04E12D517E5C000115E017EC11F082
:109ED000AA6A120EA96E03012A51A3EC01F0030134
:109EE0002B51A3EC01F003012C51A3EC01F0030171
:109EF0002D51A3EC01F0000117EC11F003012E51DC
:109F00007F5C0EE12F510001805D0AE103013051B9
:109F10000001815D05E1030131510001825D15E021
:109F200017EC11F0AA6A160EA96E03012E51A3ECCC
:109F300001F003012F51A3EC01F003013051A3EC18
:109F400001F003013151A3EC01F0000117EC11F015
:109F500082A2FED717EF11F017EC11F017EC11F0F9
:109F600001EEECF04C0EEE6E610EEE6E740EEE6EC7
:109F70003A0EEE6EEF6A17EC11F02DC32DF02CC3E4
:109F80002CF02BC32BF02AC32AF0316A306A200E42
:109F90002F6E820E2E6E33EC06F001080CE017ECEB
:109FA00011F017EC11F001EEECF0EE50FEE1ED5285
:109FB000300EEE6EEF6A17EC11F017EC11F001EEB7
:109FC000ECF0EE50FEE1ED52020E016E2DC325F0D5
:109FD0002CC324F02BC323F02AC322F098EC00F00A
:109FE000200EEE6E4C0EEE6E6F0EEE6E6E0EEE6E80
:109FF0003A0EEE6EEF6A17EC11F031C32DF030C35C
:10A000002CF02FC32BF02EC32AF0316A306A480E91
:10A010002F6E850E2E6E33EC06F001080CE017EC67
:10A0200011F017EC11F001EEECF0EE50FEE1ED5204
:10A03000300EEE6EEF6A17EC11F031C32DF030C325
:10A040002CF02FC32BF02EC32AF0316A306A200E79
:10A050002F6E820E2E6E33EC06F001080CE017EC2A
:10A0600011F017EC11F001EEECF0EE50FEE1ED52C4
:10A07000300EEE6EEF6A17EC11F017EC11F001EEF6
:10A08000ECF0EE50FEE1ED52020E016E31C325F010
:10A0900030C324F02FC323F02EC322F098EC00F03D
:10A0A000EF6A17EC11F03EA40CD017EC11F017EC8E
:10A0B00011F0200EF36E01EEECF003014A51F3CFE4
:10A0C000EBFF000117EC11F0800E016E0FEC00F0B9
:10A0D00001EEECF0EE5003E034EC01F0FBD717ECAE
:10A0E00011F0200E34EC01F0030E34EC01F0200EE0
:10A0F00034EC01F0500E34EC01F0200E34EC01F0A1
:10A10000020E34EC01F01C0EF76EE60EF66E2CEC2F
:10A1100001F0000E34EC01F0200E34EC01F0560E8C
:10A1200034EC01F0200E34EC01F0010E34EC01F0BF
:10A13000200E34EC01F017EF11F017EC11F017ECD2
:10A1400011F0AA6A040EA96EB3EC01F0646EB3ECD0
:10A1500001F0656E17EC11F017EC11F0AA6A060E0B
:10A16000A96EB3EC01F0666EB3EC01F0676E17EC0C
:10A1700011F017EC11F0AA6A080EA96EB3EC01F009
:10A180006C6EB3EC01F06D6E17EC11F017EC11F082
:10A19000AA6A0A0EA96EB3EC01F06E6EB3EC01F080
:10A1A0006F6E17EC11F017EC11F0AA6A0C0EA96E85
:10A1B000B3EC01F0706EB3EC01F0716E17EC11F0BE
:10A1C00017EC11F0AA6A0E0EA96EB3EC01F0636EE3
:10A1D00017EC11F017EC11F0AA6A0F0EA96EB3EC90
:10A1E00001F0936F17EC11F017EC11F0AA6A100E42
:10A1F000A96EB3EC01F00301496F17EC11F017ECF5
:10A2000011F0AA6A110EA96EB3EC01F00301456FBB
:10A2100017EC11F017EC11F0AA6A120EA96EB3EC4C
:10A2200001F003012A6FB3EC01F003012B6FB3ECD3
:10A2300001F003012C6FB3EC01F003012D6F17EC5B
:10A2400011F017EC11F0AA6A160EA96EB3EC01F02A
:10A2500003012E6FB3EC01F003012F6FB3EC01F09B
:10A260000301306FB3EC01F00301316F17EC11F013
:10A2700017EC11F0AA6A1A0EA96EB3EC01F00301F3
:10A28000326FB3EC01F00301336F17EC11F0020EE3
:10A290000301455DD8A4010E336E040E455DD8A4BC
:10A2A000010E33160A0E455DD8A4010E3316140EA6
:10A2B000455DD8A4010E3316000107E017EC11F03C
:10A2C00017EC11F00301040E456F000117EC11F0BB
:10A2D00017EC11F044C050F043C04FF017EC11F0F0
:10A2E00017EC11F046C052F045C051F017EC11F0D8
:10A2F00017EC11F044C054F043C053F017EC11F0C8
:10A3000017EC11F046C056F045C055F017EC11F0AF
:10A3100017EC11F003014551B40DF3CFBAF0F4CFAF
:10A32000BBF017EC11F017EC11F003014551680D6B
:10A33000F3CFBCF0F4CFBDF00001BD2717EC11F056
:10A3400017EC11F0635003014503F4CFBFF0F3CFD6
:10A35000BEF017EC11F017EC11F0030145510A0D96
:10A36000F3CFC0F0F4CFC1F017EC11F017EC11F0FF
:10A3700003014551640DF3CFC2F0F4CFC3F017ECE5
:10A3800011F017EC11F0030145511E0DF3CFC6F08B
:10A39000F4CFC7F017EC11F017EC11F003014551A1
:10A3A000320DF3CFC4F0F4CFC5F017EC11F017EC79
:10A3B00011F0030145510F0DF3CFC8F0F4CFC9F0F0
:10A3C00017EC11F00001120017EC11F0200E34EC24
:10A3D00001F0000E34EC01F0200E34EC01F04D0ED3
:10A3E00034EC01F0200E34EC01F0010E34EC01F0FD
:10A3F000200E34EC01F034EC01F034EC01F0040EEA
:10A4000034EC01F0200E34EC01F034EC01F034ECCB
:10A4100001F034EC01F0000E34EC01F0200E34ECCD
:10A4200001F0560E34EC01F0200E34EC01F0010E78
:10A4300034EC01F0200E34EC01F017EF11F017ECC2
:10A4400011F0200E34EC01F0000E34EC01F0200E7F
:10A4500034EC01F04D0E34EC01F0200E34EC01F040
:10A46000010E34EC01F0200E34EC01F034EC01F07C
:10A4700034EC01F0040E34EC01F01C0EF76EF00E1B
:10A48000F66E2CEC01F017EF11F017EC11F0FDD780
:10A4900017EC11F0FDD717EC11F017EC11F00301D8
:10A4A00045517803F3CF3FF0F4CF40F07903F350F8
:10A4B000402617EC11F017EC11F03A8017EC11F070
:10A4C00041500001BE5D4250BF594250BF19D8B043
:10A4D000800A27E617EC11F017EC11F04150BA5D35
:10A4E000416E4250BB59426E17EC11F017EC11F05F
:10A4F000BA513F26BB51402217EC11F0BC513F5CD2
:10A50000BD5140584050BD19D8B0800A0AE717EC39
:10A5100011F017EC11F0BC513F5C3F6EBD5140583B
:10A52000406E17EC11F0D2EC46F017EC11F017EC7E
:10A5300011F040C07BF33FC07AF3120017EC11F02A
:10A5400017EC11F0030145517C03F3CF80F3F4CFF6
:10A5500081F37D03F350812717EC11F017EC11F014
:10A560003A8217EC11F0030180510001BE5D030136
:10A5700081510001BF59030181510001BF19D8B0B9
:10A58000800A0FE617EC11F017EC11F0030180516F
:10A590000001BA5D0301806F81510001BB590301C5
:10A5A000816F000117EC11F017EC11F081C37FF3FC
:10A5B00080C37EF3120017EC11F00301846B030ECD
:10A5C0000301845D00012DE217EC11F003EE85F02C
:10A5D00003018451EB50076E300E075C010ED8B0BA
:10A5E000000E336E03EE85F08451EB50076E3A0E89
:10A5F000075C000102E2000E01D0010E33120BE0F5
:10A6000017EC11F017EC11F003018369826917EC64
:10A6100011F00001120017EC11F00301842B00016E
:10A62000CEE317EC11F017EC11F001EE88F016EC08
:10A6300000F00301826F18C083F30001120017ECD1
:02A6400011F017
:020000040030CA
:03000100C81F1CF9
:02000500018177
:060008000FC00FE00F40E5
:0200000400F00A
:100000006C001800F80200006C00180068065AF82E
:0C001000460484410F7E831E8FC5CC0087
:00000001FF
